:04000005000080C1B6
:020000040000FA
:108000008028002009830000118300009196000061
:10801000000000000000000000000000D53AFEDF74
:108020008F9E939B01999697FE000000B9810000F6
:1080300000000000083001005D820000BD820000E9
:108040001B8300001B8300001B8300001B830000B8
:108050001B8300001B8300001B8300001B830000A8
:108060001B8300001B8300001B8300001B83000098
:108070001B8300008D9E00001B8300001B830000FB
:108080001B8300001B8300001B8300001B83000078
:108090001B8300001B8300001B8300001B83000068
:1080A000759F00001B8300001B8300001B830000E2
:1080B0001B8300001B8300001B8300001B83000048
:1080C00000F002F800F030F80CA030C8083824188E
:1080D0002D18A246671EAB4654465D46AC4201D100
:1080E00000F022F87E460F3E0FCCB6460126334202
:1080F00000D0FB1AA246AB463343184718CD000008
:1081000038CD00000023002400250026103A01D3BA
:1081100078C1FBD8520700D330C100D50B6070473F
:108120001FB51FBD10B510BD00F040FB1146FFF795
:10813000F7FF06F06DFA00F058FB03B4FFF7F2FF0B
:1081400003BC00F05BFB000080F309887047EFF38D
:1081500009807047684680F3098806480078C007A0
:1081600003D1032080F314887047022080F3148821
:1081700070470000D8410100064B9C46EFF3058391
:108180001B0605D1EFF31483DB0701D000DF704736
:10819000604700001DF40000064B9C46EFF305838A
:1081A0001B0605D1EFF31483DB0701D000DF704716
:1081B0006047000031F60000EFF309808169891EF5
:1081C0000978002933D1A6461FC8A4467446E04763
:1081D0001F4B06CB914224D0083B002910D00CB491
:1081E000203101234B70EFF30983203B4B60F0C338
:1081F00044464D4656465F46F0C307F0AFFC0CBC04
:108200001A60203253681033F0CBA046A946B2461C
:10821000BB4683F30988203BF0CB5078002803D07D
:108220001078EFF3098318600223DB43184710B579
:10823000084A1268914209D8074C89006458A6463A
:108240001FC8A446F047EFF309840FC410BD000017
:10825000B8F4FF1F608800006088000007F064FB2E
:10826000154B06CB914223D0083B0CB420310023A0
:108270004B70EFF30983203B4B60F0C344464D46FF
:1082800056465F46F0C307F069FC0CBC1A6020320A
:1082900053681033F0CBA046A946B246BB4683F3E1
:1082A0000988203BF0CB5078002801D01078186165
:1082B0000223DB4318470000B8F4FF1F07F006FD58
:1082C000CEE7000006F050FC07F000FDC8E7000014
:1082D00070B505460C46164602E00FCC0FC5103EA1
:1082E000102EFAD2082E02D303CC03C5083E042E6A
:1082F00007D301CC01C5361F03E021782970641C27
:108300006D1C761EF9D270BD0748804707480047AC
:10831000FEE7FEE7FEE7FEE7FEE7FEE70448054965
:10832000054A064B70470000D99D0000C18000003F
:108330008026002080280020802700208027002021
:10834000004870471C260020034610B50B439B07CE
:108350000FD1042A0DD308C810C9121FA342F8D0A8
:1083600018BA21BA884201D9012010BD0020C043AB
:1083700010BD002A03D0D30703D0521C07E0002011
:1083800010BD03780C78401C491C1B1B07D10378D7
:108390000C78401C491C1B1B01D1921EF1D11846C0
:1083A00010BD000030B5441C03E00178401C0029DA
:1083B0000DD08107F9D10B4BDD0104C8D11A9143CF
:1083C0002940FAD0001B0A0603D0C01E30BD001B96
:1083D00030BD0A0401D0801E30BD0902FCD0401E11
:1083E00030BD000001010101421E5378521C002BD8
:1083F000FBD10B78491C1370521C002BF9D170472C
:10840000FFFFFFFFFFFFFFFFFFFFFFFFFEFFFFFF7D
:108410000346F0B50B439B072DD1244DEF01042AF1
:1084200029D308C810C95E1B9E43121F3E4017D0B7
:10843000D8B2E1B2401A3106014310D198B2A1B2CC
:10844000401A310401430AD118022102000A090A24
:10845000401A3102014302D1180E210E401AF0BD1C
:10846000A342DCD018BA21BA884201D90120F0BD5C
:108470000020C043F0BD002A01D10020F0BD0378E8
:108480000C78401C491C002B0DD0A3420BD1521E6E
:1084900009D003780C78401C491C002B03D0A34260
:1084A00001D1521EEBD1181BF0BD000001010101EA
:1084B000F8B5042A2CD3830712D00B78491C03701B
:1084C000401C521E83070BD00B78491C0370401CC4
:1084D000521E830704D00B78491C0370401C521EA7
:1084E0008B079B0F05D0C91ADF002023DE1B08C9AC
:1084F0000AE0FFF7EDFEF8BD1D4608C9FD401C4629
:10850000B4402C4310C0121F042AF5D2F308C91A34
:10851000521EF0D40B78491C0370401C521EEAD442
:108520000B78491C0370401C012AE4D409780170BF
:10853000F8BD431A70B593421BD28918801804E025
:10854000491E401E0B78521E03709307F8D106E0B7
:108550001039103878C9103978C01038103A102AFC
:10856000F6D203E0091F001F0B680360121FF9D544
:1085700070BDFFF7ADFE70BDF8B506461446084362
:10858000800707D0751AA54219D20819102D13D2E9
:10859000311907E03046FFF7CCFFF8BD401E491EF9
:1085A00002780A70641EF9D2F8BD471B2A46394684
:1085B000FFF77EFF641B3846A542F6D3011B224617
:1085C0003046FFF775FFF8BDD2B210B513029A1806
:1085D00013049A1800F00EF810BD01E004C0091F42
:1085E0000429FBD28B0701D50280801CC90700D06B
:1085F0000270704700290BD0C30702D00270401CE4
:10860000491E022904D3830702D50280801C891EDB
:10861000E3E70022EEE70022DFE70378C27819469D
:10862000437812061B0219438378C0781B04194350
:1086300011430902090A000608437047020A08703C
:108640004A70020C8A70020ECA7070470022030939
:108650008B422CD3030A8B4211D300239C464EE05D
:1086600003460B433CD4002243088B4231D3030919
:108670008B421CD3030A8B4201D394463FE0C309CB
:108680008B4201D3CB01C01A524183098B4201D3E3
:108690008B01C01A524143098B4201D34B01C01ACE
:1086A000524103098B4201D30B01C01A5241C30846
:1086B0008B4201D3CB00C01A524183088B4201D3B5
:1086C0008B00C01A524143088B4201D34B00C01AA1
:1086D0005241411A00D201465241104670475DE0B6
:1086E000CA0F00D04942031000D340425340002239
:1086F0009C4603098B422DD3030A8B4212D3FC22E2
:10870000890112BA030A8B420CD3890192118B4260
:1087100008D3890192118B4204D389013AD0921176
:1087200000E08909C3098B4201D3CB01C01A524131
:1087300083098B4201D38B01C01A524143098B42FA
:1087400001D34B01C01A524103098B4201D30B01E3
:10875000C01A5241C3088B4201D3CB00C01A524108
:1087600083088B4201D38B00C01A5241D9D24308EF
:108770008B4201D34B00C01A5241411A00D201462C
:10878000634652415B10104601D34042002B00D596
:108790004942704763465B1000D3404201B5002058
:1087A000C046C04602BD7047704770477546FFF728
:1087B000C7FDAE46050069465346C008C000854661
:1087C00018B020B5FFF7AAFD60BC00274908B646DF
:1087D0000026C0C5C0C5C0C5C0C5C0C5C0C5C0C5D0
:1087E000C0C5403D49008D46704710B50446C0469F
:1087F000C0462046FFF7A1FC10BD0000014918202B
:10880000ABBEFEE726000200704770B58C180578F5
:10881000401C6B075B0F01D10378401C2A1106D165
:108820000278401C03E00678401C0E70491C5B1E59
:10883000F9D12B0705D40023521E0DD40B70491C0F
:10884000FAE70378401CCB1A921C03E01D780D70E8
:10885000491C5B1C521EF9D5A142D8D3002070BD23
:1088600000000000F8B502787F2A02D000F04EF830
:10887000F8BD0A704478861C4C708D1C074F08E0C8
:108880002946304600F042F8010C3F188E1980B29C
:108890004519641EF4D23846F8BD000002000200FB
:1088A0000A4670B5014600200346062916D006DCAC
:1088B0000B0003F0DDFF0513131314181300FD293B
:1088C0000CD003DCF02909D111201CE0FE2919D0BD
:1088D000FF2903D1402010705370022070BD15464F
:1088E00005F02AFD02E0154605F02EFD0646FFF7CD
:1088F00059FD401CC4B2224631462846FFF7D8FD38
:10890000204670BD05201070012070BDF8B50278BA
:108910001346803B1F2B02D800F02AF9F8BD1346FE
:10892000A03B5E2B02D800F0A9F9F8BD0A700778C9
:108930004C1C421C0025FF218548864E3B0003F05D
:1089400097FF1E1018213EA6B3D0F2EB4F61F2F252
:10895000F2F2F2656A6F7E8DA33BF2F2F2F2F2F26E
:1089600088F21078611CFFF79BFF7B49207040184C
:10897000F8BD1078002843D0012841D021707648F6
:10898000401ECEE01178002903D0012902D0002139
:1089900012E001210122027070482025456040222A
:1089A00042600223436047692F434761456915438D
:1089B000456142691A43426121703046B1E0057059
:1089C0006648426920218A434261426940218A43C4
:1089D0004261426902218A43426125700120A0E080
:1089E0005078117807025F480F435D490068FFF730
:1089F0002DFE0321801CFFF729FE7843401EFDD188
:108A00002570BCE76570257002208AE0214610467B
:108A100000F0D2FB85E02146104600F09DFB80E08F
:108A20001778511C002F01D1FF270137384601F07C
:108A3000ADF9FF1D2570F8080004801971E0117868
:108A40008A07920F521C49070276C90F417625709A
:108A5000B3E72146104600F017F962E021700121CA
:108A600013780C46521C0AE01078521C8006800EC7
:108A700000D14020C01DC00812180918491C5B1EF7
:108A8000F2D2080420434CE010782170D4E711782A
:108A90000173937857781902394301821179D2789A
:108AA0000902114341824DE000782146012814D08B
:108AB0001346521C1078521C002808D01778521CFC
:108AC000BC0701D5FC0600D5121D401EF6D1D01AF8
:108AD0000D7000044D70801C23E0104600F018F962
:108AE0001FE0007817462146012809D00D704D700F
:108AF000A5700320F9781C4A890705D5104310E0BA
:108B0000104600F097FAF5E7B9787B780902194327
:108B100089048918084304E00078012804D02170F2
:108B200012488019F8BD0FE01746501CFFF775FD7D
:108B300039790002000A09060843009069460020BE
:108B400000F09AFE2570EBE7203CE1773046E9E73C
:108B5000F0F5FF1F010001000200020080F00F404D
:108B600040420F00D8F2FF1F000004000100050082
:108B7000FEB502780A704D1C01783D4C401C8039CE
:108B80000646671C0B0003F073FE0D0816223840E2
:108B90007171714755606468710005F0CDFB07463F
:108BA000FFF700FCC6B22E70681C32463946FFF74C
:108BB0007FFCA41927E00724684601F017FC224631
:108BC00069462846FFF774FC294C08344EE0684695
:108BD00001F00CFC002002900422314602A8FFF7AD
:108BE00067FC02980090684601F020FC002001F02C
:108BF0009DFC012028701F4C38E03E21681C08F0C5
:108C000039FE28702418641C30E03778401C39463F
:108C100008F094FE012025E001202870307800281B
:108C200005D0012803D000202870134C1EE005F069
:108C30009BFEFAE70120287004F046F8002802D1D4
:108C4000022008F0E1FB3C4610E0007807F0BCFA97
:108C5000EAE707F085FA2870F5E73778401C3946CF
:108C600007F054FB28703904081904192046FEBD8A
:108C7000010001000200050002000200FF20087050
:108C80000048704701000100F3B583B000220A706C
:108C9000491C0125009504910178441C01912AE0AA
:108CA0002778641CB806800E00D14020C01DC6087D
:108CB00038061648416902D54022914301E040221E
:108CC0001143416121463846049A00F089FD01981C
:108CD000002804D10D484169402211434161380602
:108CE00006D504988019049000988019009001E03E
:108CF000A419AD196D1C0198401E0190401CCFD1E4
:108D000000992804084305B0F0BD000080F00F4032
:108D1000F0B589B00890044600208D1C0391C3492A
:108D200002900870049005906678A41C002E6FD005
:108D30002778641CB9076CD50499002935D0BC4844
:108D4000008A01901120384001280FD16946384629
:108D500000F092FD02281AD10199491E0191491C87
:108D600003D0B24909780029F0D012E169460E20FB
:108D700000F082FD022808D10199491E0191491C89
:108D800003D0AA4909780029F0D0002104910128D4
:108D9000EBD1009929700099090A69700099090CB2
:108DA000A9700099090EE9702D1DF90658D52046C5
:108DB000FFF733FCE1780002000A09060843079038
:108DC0009B48241D408A0690F80715D09848008AD1
:108DD00001900021384600F04FFD022802D0012802
:108DE000C3D109E00199491E0191491CBDD08F49A9
:108DF00009780029EDD0CCE08D48008A01906946C1
:108E0000384600F039FD022804D001281CD10BE0BF
:108E1000E0E064E00199491E0191491C14D08349A6
:108E200009780029EBD00FE08149009A4969114087
:108E3000079A914208D00699491E0691491C03D011
:108E40007A4909780029D7D07949009A49691140AF
:108E5000079A914201D01021084301281AD13CE021
:108E60007349098A0191F90718D00499002934D16E
:108E70000021384600F000FD022802D0012809D167
:108E800009E00199491E0191491C03D067490978FD
:108E90000029EDD07DE0012104911EE069463846AD
:108EA00000F0EAFC022802D0012872D109E0019901
:108EB000491E0191491C6CD05C4909780029EDD00C
:108EC00067E0009929700099090A69700099090CF6
:108ED000A9700099090EE9702D1D00214DE004983C
:108EE000002823D05248008A019069460E2000F0E5
:108EF000C3FC022802D001284BD109E00199491E88
:108F00000191491C45D0494909780029EDD040E03C
:108F1000009828700098000A68700098000CA870EB
:108F20000098000EE87000202D1D04902046FFF7E9
:108F300074FBE1780002000A09060843241D009032
:108F4000B90603D53A494861012017E03848008A3C
:108F500001906946384600F08FFC022802D00128B3
:108F600017D109E00199491E0191491C11D02F49DF
:108F700009780029EDD00CE0012105910299491CE6
:108F800002912A490978002903D1761E00D0CFE644
:108F90000AE0002E08D02178641C8A0701D5C90692
:108FA00000D5241D761EF4E7012832D1049900294A
:108FB0001ED01F481D4F068A69460E2000F05CFC3B
:108FC000022802D0012824D105E0761E21D3397869
:108FD0000029F1D01DE0009929700099090A6970F3
:108FE0000099090CA9700099090EE9702D1D10E077
:108FF000059900290DD00E480C4F068A00210E203D
:1090000000F03AFC022804D1761E02D339780029F8
:10901000F4D0039A02991170039948700898039943
:10902000201A0004691A084309B0F0BD00F0FF1FC0
:10903000F0F5FF1FF3B583B00025CE1C0291444923
:10904000024628460D70917853780C02D21C1C43BE
:1090500073D01178521C0091039289075DD5009955
:10906000C90737D03B48078A0021009800F004FC6C
:10907000022802D0012860D12CE07F1E5DD3344944
:1090800009780029F0D058E0002C04D10098C007DE
:1090900001D00E2000902F48078A01A9009800F007
:1090A000EBFB022802D0012847D106E07F1E44D303
:1090B000274909780029F0D03FE0019931700199E2
:1090C0006D1C090A71700199090CB1700199090EA2
:1090D000F170361D641ED7D22FE00398FFF79DFA7A
:1090E00003990002C978000A090608430190039811
:1090F000001D03901748078A01A9009800F0BCFBE7
:10910000022802D0012818D106E07F1E15D310498D
:1091100009780029F0D010E06D1C641EDDD20D48E6
:109120000B4F048A00210E2000F0A6FB022804D178
:10913000641E02D339780029F4D002990D70029A86
:10914000290A517002998870029805B0301AF0BD52
:1091500000F0FF1FF0F5FF1FF8B50C460546FFF7BE
:109160005CFA0102E878090A0006104F014309D0B1
:109170000F48002600680F4D4008884205D801209E
:1091800068700FE0FF2020700EE040186E70401EE7
:10919000FFF75CFA012804D90321401CFFF756FAB7
:1091A00000E00120686026703846F8BD0100040028
:1091B000D8F2FF1FF0F5FF1FF8B507460578447891
:1091C0000E46801CFFF729FA01027879090A000689
:1091D00001432948E20706D0EB072022002B01D0EB
:1091E000426000E08260A20706D5AB074022002B58
:1091F00001DA426000E08260220607D5EA09D3075F
:109200000222002B01D0426000E08260002923D0BE
:1092100001230022E10704D001698906C90FA94290
:1092200017D1A10705D501696F084906C90FB942D1
:109230000FD1610701D5A9080BD1A10601D5690994
:1092400007D1210608D50169EF098907C90FB9427D
:1092500002D051429942DDD3016902698906C90FE2
:109260005206D20F5200006911438007C00FC0019F
:10927000014331700148F8BD80F00F400100060045
:1092800070B5194C0025257019486570174900689C
:10929000FFF7DCF9401E6060257364202082658240
:1092A00001206561207613486576816B1F2252028A
:1092B00011438163FF201049033048610F48202289
:1092C0004260436913434361FF2404348C614022AC
:1092D00042604369934343614C60022141604269AB
:1092E0000A43426170BD0000F0F5FF1F80969800B0
:1092F000D8F2FF1F0080044000B0044080F00F400F
:10930000F8B5C41D0546F934E06C1E460F4600282A
:1093100023D0402A00DD4022401EE064606D8001C1
:109320004019FFF7C5F8606D800141193846FFF715
:1093300099FA616D49004919FF3141310880606D2A
:109340000521800140193060606D401CFFF77EF9F7
:109350006165206D401C20650120F8BD10B5C41D5D
:10936000F934236D002B17D05B1E2365A36D9B0181
:109370001B180B60A16D49000818FF3041300088B0
:109380001060A06D0521401CFFF760F9A165E06C3D
:10939000401CE064012010BD002010BDFF30002201
:1093A00001304265826505210265C1647047000095
:1093B00070B50546EFF31080C407E40F72B6094E8E
:1093C000094B29463046F26800F010F8002805D114
:1093D000002329463046F26800F0D4F8002C00D172
:1093E00062B670BDC80D00206B66656BFFB589B0B5
:1093F00016460C466A46099804F06EFC3246214631
:10940000049B099804F09DF905002BD1009C019F55
:10941000A619761E39463046FFF718F900291BD0E9
:10942000401C7843461E17E021020920090A000665
:1094300009180D4841600C9804F09CF9002811D1DE
:10944000099804F0A1F9054609980069002800D0A0
:109450008047002D02D1E419B442E5D9099804F0FF
:1094600043F928460DB0F0BD0000024070B504007D
:1094700027D01648C0680001000F0F2823D01449D8
:109480004000085A80020025256060600120A0602D
:109490006561A56180022561E060204604F043F922
:1094A00000280AD00B4801468039056041604031F0
:1094B0008160E061204600F00FF8256200206562BF
:1094C00070BD042070BD01204004DCE740800440F2
:1094D000503F01007C0E002010B500280AD0C4695E
:1094E000606803F0C5FDA06803F07EFD02202060E7
:1094F000002010BD042010BDFFB589B01F46140028
:109500000D460DD06A46099804F0E6FB3A46294616
:10951000039B099804F015F9060002D1009D28E08C
:1095200004200DB0F0BD02CC1548816003990429D8
:1095300002D0082907D00EE029020322090A5206A8
:109540008918416007E002CCC16029020722090A9C
:10955000120689184160099804F016F90646099820
:109560000069002800D08047002E04D103984519D7
:109570003F1A002FD7D1099804F0B6F83046D0E74B
:1095800000000240FFB589B014460D466A460998AE
:1095900004F0A2FB22462946059B099804F0D1F865
:1095A00000282FD16A462946099804F095FB009DB2
:1095B000029808906942404201404F42AF4201D1B7
:1095C00008983F18002C1CD07E1BA64200D92646C6
:1095D00030460599FFF73AF829020122090A1206D6
:1095E0008A1809494A600C9A000412021043FF309D
:1095F0008860099804F0C8F8002803D1A41BAD19AD
:10960000DEE700200DB0F0BD00000240FFB589B0DC
:10961000129F1D0016460C4610D06A46099804F0A9
:109620005BFB32462146079B099804F08AF8002824
:1096300005D1154A39068F18009C22E004200DB090
:10964000F0BD21020120090A400609180F484160B7
:1096500087602968C160099804F096F8002809D04D
:109660001399002900D00C6014990029E7D000223A
:109670000A60E4E70799761A890889004D19079965
:109680000C19002EDDD1DAE7FFFFFF0000000240D9
:10969000EFF3088470460007000F0D2801D1EFF3A7
:1096A00009842546A08B2035800500D52D1D7046E8
:1096B000C00600D44835704603F074FBEFF3098010
:1096C00003F070FBEFF3088003F06CFBEFF3148002
:1096D00003F068FB284603F065FB606903F062FB5A
:1096E000A06903F05FFBE06903F05CFB4A2203A181
:1096F000002003F041F900F0BBFBFEE72E2E5C2EAC
:109700002E5C2E2E5C736F757263655C6461706C89
:10971000696E6B5C486172644661756C745F486128
:109720006E646C65722E630010B5EFF31080C00795
:10973000C00F72B60021064A1160002800D162B63F
:109740000448FFF793FE002800D0012010BD000060
:1097500000810440C80D00201CB507F033F8002834
:109760001AD09E2069460870E7204870102000F04B
:109770000DFB012407F026F800280DD000206946D3
:109780000870082000F002FB01A9002006F0B0FFDD
:10979000012802D1002C00D01CBD00201CBD0000FF
:1097A000FEB5074616460D46EFF31080C407E40FDA
:1097B00072B60B4639460948FFF79EFE002809D1CC
:1097C000012101900091029033462A463946034810
:1097D000FFF71CFF002C00D162B6FEBDC80D0020B3
:1097E000F0B583069B0E00D14023224C00062026B4
:1097F0001F4D646800281BDB37E00021082012E0C1
:10980000AE601C4C646827467F1EFDD12F696E60D8
:109810007F06FF0F641EFDD14C08F9012143401E55
:109820005B1E002801D0002BEAD1C1401170521CF0
:10983000002BE2D1F0BD0A780827491C12E0D007BE
:1098400002D04020686001E04020A860AE60204661
:10985000401EFDD16E602046401EFDD152085B1EA9
:109860007F1E02D0002BEAD1F0BD002BE3D1F0BD6A
:1098700080F00F40F0F5FF1F10B5054A5278002A1E
:1098800002D000F007F810BD00F0F2F810BD0000A3
:10989000F0F5FF1FF0B5744F40228C467A6020210E
:1098A000B9607960C30701D07A6000E0BA60B9603E
:1098B00079604308DD0701D07A6000E0BA60B960E2
:1098C0007960C4188308DD0701D07A6000E0BA60CF
:1098D000B9607960E418C308DD0701D07A6000E060
:1098E000BA60B9607960E318DB0701D07A6000E004
:1098F000BA60B9607960BA60B96079607A60B9605D
:1099000079607B69402293437B61584A127E131E23
:1099100003D0B9607960521EFBD1B9603A697960B1
:109920005206D20FB9603C6979606406E40F6400A6
:109930001443B9603A6979605206D20F920022430B
:10994000012A10D0022A6DD0042A6BD0213303D013
:10995000B96079605B1EFBD1796940200143796170
:1099600078601046F0BD840727D5002425462023C3
:10997000B9603E6979607606F60FAD196408F6079E
:1099800034435B1EF4D1B9603B6979605B06DB0F41
:109990005D40EB0700D008226346002B00D01C601E
:1099A000324B1B7E002B03D0B96079605B1EFBD16C
:1099B0007B69402423437B6123E0002B03D0B96003
:1099C00079605B1EF9E77B69402633437B61634620
:1099D0001B6800252024DE0702D040267E6001E0BF
:1099E0004026BE60B9607960ED185B08641EF2D154
:1099F000EB0702D040237B6001E04023BB60B960ED
:109A00007960000602D51948002383601748007B5F
:109A1000002805D04023BB60B9607960401EFBD1AF
:109A200040209DE7114C657E002D06D0840704D5AB
:109A30002124B9607960641EFBD1002B03D0B9608A
:109A400079605B1EF9E77C6940231C437C61002D33
:109A500007D0800705D4BB602120B9607960401E23
:109A6000FBD17B607DE7000080F00F40F0F5FF1F29
:109A7000F3B50023C34E402272602024B460C24F6D
:109A800079680D466D1EFDD174600D466D1EFDD1C9
:109A9000C50701D0726000E0B260B4600D466D1E73
:109AA000FDD174600D466D1EFDD11D184308DF0702
:109AB00001D0726000E0B260B4600F467F1EFDD13D
:109AC00074600F467F1EFDD1ED188308DF0701D0BB
:109AD000726000E0B260B4600F467F1EFDD174601A
:109AE0000F467F1EFDD1ED18C308DF0701D072605D
:109AF00000E0B260B4600F467F1EFDD174600F4677
:109B00007F1EFDD1EB18DB0701D0726000E0B26070
:109B1000B4609D4D0B465B1EFDD174600B465B1E11
:109B2000FDD1B260B4600B465B1EFDD174600B4684
:109B30005B1EFDD17260B4600B465B1EFDD174608C
:109B40000B465B1EFDD173694022934373612B7EEC
:109B50001D1E09D0B4600A46521EFDD174600A462B
:109B6000521EFDD15B1EF5D1B4600A46521EFDD1D6
:109B7000326974605206D20F0B465B1EFDD1B46091
:109B80000B465B1EFDD1336974605B06DB0F0F462D
:109B90007F1EFDD15B001343B4600A46521EFDD107
:109BA00032695206D70F202272600A46521EFDD13A
:109BB000BA001A43012A17D0022A70D0042A6ED0A4
:109BC00021350AD02023B3600846401EFDD17360C2
:109BD0000846401EFDD16D1EF5D17169402001433C
:109BE000716170601046FCBD83073ED50024254698
:109BF00020232027B7600F467F1EFDD137697F06DF
:109C0000FF0FBC46202777600F467F1EFDD16708F7
:109C10006446E4073C4365445B1EEAD12023B360FD
:109C20000F467F1EFDD1376973607F06FF0F491E07
:109C3000FDD17D40E90700D008220199002900D01C
:109C40000C6051490C7E002C0AD04D68B360294647
:109C5000491EFDD173602946491EFDD1641EF5D110
:109C600071694024214371613AE0002D0AD020241B
:109C7000B4600B465B1EFDD174600B465B1EFDD1CC
:109C80006D1EF5D17369402423437361019B002746
:109C90001B682025DC0703D04024746002E038E014
:109CA0004024B4602024B4600C46641EFDD12024FE
:109CB00074600C46641EFDD1FF185B086D1EE9D16F
:109CC000FB0702D04023736001E04023B3602024EF
:109CD0003546B4600B465B1EFDD16C60491EFDD15C
:109CE000000602D5284900208860274B197B0029EF
:109CF0000DD04020B0605B682024B4601846401E40
:109D0000FDD174601846401EFDD1491EF5D140209A
:109D100067E71D4B5B7E9C46002B0DD083070BD560
:109D200021242027B7600B465B1EFDD177600B46D0
:109D30005B1EFDD1641EF5D1002D0AD02024B46035
:109D40000B465B1EFDD174600B465B1EFDD16D1E84
:109D5000F5D1746940231C4374616446002C0ED015
:109D600080070CD4B36021242025B5600846401E2E
:109D7000FDD175600846401EFDD1641EF5D17360AB
:109D800030E7000080F00F40F0F5FF1FF0B5002332
:109D9000104C1A460E4E2027656815E0002A02D1A5
:109DA0000B780822491CDC0702D04024746001E0D3
:109DB0004024B460B7602C46641EFDD177602C4609
:109DC000641EFDD15B08521E401EE7D2F0BD0000AC
:109DD00080F00F40F0F5FF1F1E48002202601E4871
:109DE000816B4315194381631B491C48403148600E
:109DF0001B4883681B490B408360C3680B40C360EA
:109E0000194980200870194824214170A22101704D
:109E1000C178C906C90EC1700321017142718179EF
:109E2000C906FCD481790907890F0229FAD140219A
:109E3000417181790907890F0229FAD1817949068F
:109E4000FCD51A21017081790907890F0329FAD1FC
:109E500070470000008104400080044000000110B1
:109E600040900440FFF8FFFE0050064000400640CE
:109E7000BFF34F8F04490348C860BFF34F8F00BF43
:109E8000FDE700000400FA0500ED00E038B5254DBF
:109E90002C79E878800601D420208443E8780006F5
:109EA00001D480208443200616D51F4802F009FE05
:109EB000002800D00120E7221CA102F05DFD1A4815
:109EC00002F020FEE871184802F0FBFD002803D1E3
:109ED000E8784006400EE870A00605D56007800FC0
:109EE00003D0E8796946087038BDED791B4802F067
:109EF000D7FD0446132804D92946184802F03EFE2F
:109F000038BD02F0F1FE002807D0132CF8D113223F
:109F100013A1124802F083FE38BD104802F0F2FD92
:109F2000EAE7000000B00640880E00202E2E5C2ECE
:109F30002E5C2E2E5C736F757263655C6869635F5F
:109F400068616C5C667265657363616C655C6B6CA3
:109F500032367A5C756172742E63000098100020AE
:109F60003C4441504C696E6B3A4F766572666C6F3B
:109F7000773E0A00F8B52E4E002435780095280764
:109F800041D5317C0A090807C00F4B07DB0F154686
:109F900005431AD1950040002818C018254BC00071
:109FA0001D5CAD062D0F012D0FD1C5186F88002F38
:109FB0000BD1214FBA5C6A801A5C520601D5882207
:109FC00000E0C8221A5401200143EFF31080C507B6
:109FD000ED0F72B6194A184F143FB8681154192181
:109FE000401CFEF733FBB960002D00D162B608209B
:109FF0003070002C02D1307D800601D5012400E0B4
:10A0000000243578BBE700990B482943083804F051
:10A01000B6FF002C01D0012000E0002006491439D1
:10A020000A7810430870357002F0CEFBF8BD0000CE
:10A0300080200740001600209CF4FF1FC01C002059
:10A040001CB5002001906A4601A90948FFF786F96E
:10A05000002808D0074880210078009A0843019919
:10A0600002F0DAFB1CBD0449012008701CBD000091
:10A0700038230020963F010018F5FF1F38B5174D13
:10A08000174C28886188421A16486168007801F0E8
:10A0900053FF616880B209186160618809188AB24B
:10A0A000628029888A4206D20F49104B09784900FC
:10A0B000595A814211D96B460D490E48FFF720F9D4
:10A0C0000025002806D02078002803D00020FFF7C4
:10A0D000B7FF257065800648606038BD9C3F010071
:10A0E00018F5FF1F973F010063F5FF1F983F010020
:10A0F000F21400203823002010B50446400702D592
:10A100000020FFF7BBFF200702D50020FFF798FFD4
:10A1100010BD002070470000034801694069081A1B
:10A1200002490988081A704720F5FF1F8C3F01007B
:10A1300070B50B4D0C460346696B286B88420BD9F2
:10A14000401A844200DD044622461846FEF7B0F964
:10A15000686B0019686300E00024204670BD0000B1
:10A1600020F5FF1F00207047F8B5184F0C46064633
:10A1700079693869401A16490988081A002801DCEB
:10A180000020F8BD844200DD0446FA69B869002564
:10A1900090420DD30F4A031951188B4208D30D1A60
:10A1A0002A463146FEF784F976190A48641BB861DD
:10A1B000002C06D022463146FEF77AF9B86900191C
:10A1C000B8613969601909183961F8BD20F5FF1FB8
:10A1D0008C3F01007214002010B5054C6068002807
:10A1E00005D10120606000F005F80020606010BD1E
:10A1F00020F5FF1FF8B5234CA06800283DD0616909
:10A2000020690026421AE06811460143002935D032
:10A2100021461D4FC9691D4D002A10D0A0698142F9
:10A2200005D338888B182818834200D3421A18485F
:10A23000007843001748C05A904200DA0246164898
:10A24000E66000788023184302F0E6FAE169091815
:10A25000E1616269121862613B88EB188B4200D1A0
:10A26000E561216991420BD1094909784A00094900
:10A27000895A814204D10120E060F8BDA660F8BD92
:10A28000E660F8BD20F5FF1F8C3F0100721400202E
:10A2900063F5FF1F903F01008A3F010010B50C4C91
:10A2A000206A002803D0A06A401CA06210BD0120D3
:10A2B0002062606200F00EF8002060622062616B34
:10A2C000206B8842F2D0401AFFF74CFF10BD00000F
:10A2D00020F5FF1F10B5134C1348216B154B0A1ABC
:10A2E00012480088821A124800784000185A8242A8
:10A2F0000EDB1148007801F01FFE216B0818206367
:10A30000A06A00280CD0616A002909D1401E06E02D
:10A310000120E062606A002802D0A06A401CA062AE
:10A3200010BD000020F5FF1FB21400208E3F010079
:10A3300063F5FF1F903F01008B3F010010B50446FD
:10A34000400702D52046FFF7A9FF200702D5204687
:10A35000FFF742FF10BD7047002070470020704794
:10A3600010B50C4800F042F8002812D00948FEF75A
:10A3700054F90949020A08704A70020C8A70000EEA
:10A38000C870044802790A7142794A7180798871EB
:10A39000012010BD58F5FF1F7013002010B51048A4
:10A3A000002444608460C46004610E49816144619A
:10A3B000046244628462C462C1610B490163416307
:10A3C000014604804B203831C001FEF737F90448BC
:10A3D0000821383004714471817100F019F810BD02
:10A3E00020F5FF1F72140020B214002070B504463F
:10A3F000064D21462868FEF721F92879A071687971
:10A400006071A8792071012070BD0000E8F5FF1F80
:10A4100010B507F0FBF904F027F9012010BD10B5C5
:10A4200007F032FA012010BD0120704710B5044634
:10A43000FEF7F3F806490860A07908716079487161
:10A44000207988710020C871084607F02FFA10BDE6
:10A45000E8F5FF1F10B51148002444608460C46013
:10A4600004610F4981614461046244628462C46290
:10A47000C1610C49016341630480FFF7D0FF0749C4
:10A480004B203831C001FEF7D9F804480821383094
:10A49000047144718171FFF7C9FF10BD20F5FF1FE2
:10A4A00072140020B214002010B5FFF7D3FF10BDC6
:10A4B00070B51B480078002831D01A4C0025206A5E
:10A4C000012600280AD1616B206B884206D116490B
:10A4D000884203D02163E56225626163A06A002897
:10A4E00010D0206A00280DD1E06A00280AD1266227
:10A4F000FFF7F0FE2562616B206B884202D0401AA4
:10A50000FFF730FEA1686068084308D161692069DF
:10A51000884204D06660A660FFF76CFE656070BD7F
:10A5200061F5FF1F20F5FF1FB214002070B505462E
:10A530000F480068C1698847002816D10D4C002DCE
:10A5400006D004F033FA2060002006F05DFF0CE036
:10A5500004F02CFA2168401AFF212D31884201D3E2
:10A56000012000E0002004F089F8012070BD000007
:10A5700050310100E4F5FF1F0020704700207047B4
:10A5800010B502490880FFF74FFF10BD20F5FF1FEF
:10A5900010B50B48FEF741F8094C0002E178000ABB
:10A5A000090608430749FEF749F806482179017171
:10A5B00061794171A1798171FFF738FF10BD000009
:10A5C0007013002058F5FF1F01078A0E044910B5CB
:10A5D00051180A78FD231A400A7002F08FF810BD56
:10A5E000C020074010B501464A790B7980781102E6
:10A5F0001943020601D4024A115402F07FF810BD3B
:10A600009CF4FF1F704710B500F016FB10BD000052
:10A61000094A094980320028087D04D001231843E3
:10A620000875102005E0400840000875107AEF21F9
:10A6300008401072704700008020074010B50C4C95
:10A640000C48A2880078824200D90246002A03D131
:10A6500007490020143908718020216802F0DCF8D5
:10A66000216809182160A188081AA08010BD000087
:10A6700074F5FF1F713F010010B5064C0020A28841
:10A68000216801F059FC216809182160A188081A85
:10A69000A08010BD74F5FF1F704700000749020637
:10A6A00005D50007800E40180178FA2203E08000EB
:10A6B00040180178F622114001707047C020074011
:10A6C0000749020605D50007800E401801780522CB
:10A6D00003E080004018017809221143017070479F
:10A6E000C0200740F8B504466F4F704D704E80078C
:10A6F00020D502F05FF83878C009FFF7CDFFF88861
:10A70000A88038784106890F04D001295CD002293D
:10A7100075D169E079780B0002F0AAF80C070D7189
:10A7200013711928712D333B4A7101F0ABFD1FE005
:10A73000FFF784FF70E0002004E002F04FF85D486E
:10A740003DE0012001F0E0FD002858D0F5E7C0060B
:10A75000C00E54D1B8788021084330704006400EB6
:10A76000012102F011F802F039F855E001F074FC13
:10A77000002844D0DCE7C006C00E40D14C48401C45
:10A7800014E001F015FE002839D002F027F84A48FD
:10A7900015E0C006C00E012831D1707800282ED0F7
:10A7A0003879B17888422AD2444940182860BFE7F6
:10A7B00001F0C2FE002822D002F010F840480068E4
:10A7C000002829D0804727E0C006C00E17D00128F6
:10A7D00015D100F017F900281ED100F06FF90028FC
:10A7E0001AD100F0BBF808E0C006C00E07D100F097
:10A7F0009FF9002810D100F0E7F900280CD1387833
:10A80000C00904D1F888002801D0002000E0802091
:10A8100001F0C4FF0020A880600704D53878C00983
:10A820000DD001F0E3FF200733D53878C00927D0D9
:10A83000A888317908432CD0FFF700FF29E0A888C9
:10A840000028F0D0FFF718FFA8880028EBD138784F
:10A850004106890F0ED001290CD1C006C00E09D0C7
:10A86000012807D100F05CF80028DCD100F02AF8BC
:10A870000028D8D1802001F091FF0020A880D2E7E5
:10A880003078010605D54006400E3070002101F0F9
:10A890007BFF600602D50020FFF796FE200602D55A
:10A8A0008020FFF791FEF8BD7CF5FF1F74F5FF1FB8
:10A8B00060F5FF1FFC3F0100F43F010077F4FF1F2C
:10A8C000F83F010010B51349134A087912789042F5
:10A8D00003D0124A1278904219D14878002804D047
:10A8E000022805D0202812D10EE0FFF745FE05E032
:10A8F000C878897800020843FFF740FE002806D098
:10A9000001F06CFF012010BDFFF742FEF6E70020CA
:10A9100010BD00007CF5FF1FDCF2FF1FDDF2FF1F02
:10A9200010B50B490B4A08791278904203D00A4AB5
:10A93000127890420AD14878092807D100F082FBAA
:10A94000002803D001F04AFF012010BD002010BDF7
:10A950007CF5FF1FE0F2FF1FE2F2FF1F70B52449F4
:10A96000244A08791278904203D0234A1278904200
:10A970003BD11F484978C278837810021F4C204D84
:10A980001843042920D008DC00290FD001290FD05A
:10A9900002290BD0032928D111E0202906D0212932
:10A9A00019D022291AD023291FD11AE02C6010E0D7
:10A9B000FFF7D4FC05E02C60FFF740FE09E0FFF74D
:10A9C000CBFC0028F7D110E0FFF7A3FB0BE001F070
:10A9D00005FF012070BDFFF7C3FCF2E7FFF7D0FDD4
:10A9E00001E0FFF7A3FD0028F1D1002070BD0000B9
:10A9F0007CF5FF1FDCF2FF1FDDF2FF1F701300204C
:10AA000074F5FF1FF8B5254E25493079097888423D
:10AA100003D02449097888423DD17078224C234DD7
:10AA2000234F030001F024FF0C3707232D3737375E
:10AA300037371826333700F023FA00282BD0F07868
:10AA4000012802D0032803D003E01A48206000E068
:10AA50002560FFF7F3FD12E0F078022802D003280A
:10AA600003D00CE01448206009E0256007E000F006
:10AA7000EFF908E000F0BEFA0BE001F0AFFE0120B4
:10AA8000F8BD00F0F3F9002805D02760E1E700F0F9
:10AA9000CFFA0028F1D10020F8BD00007CF5FF1F9F
:10AAA000E0F2FF1FE2F2FF1F74F5FF1F84F4FF1FA7
:10AAB00070130020B1130020F213002010B51848C5
:10AAC000184A01791278914227D142780146C87814
:10AAD0008B7800021843CB798C7919022143FE2A26
:10AAE0000CD0FF2A19D1002817D1002915D101F067
:10AAF00063F9002811D001F071FE0CE000280CD1A0
:10AB000001290AD100F048FE002806D0074906486E
:10AB10000860FFF793FD012010BD002010BD00006C
:10AB20007CF5FF1FE1F2FF1F7013002074F5FF1F7B
:10AB300070B51F4D1F49687809780026884235D1C5
:10AB4000687929790002084302282FD1AA781A4C83
:10AB5000002A2BD0002004E02178002900D00C1915
:10AB6000401C411C8A42F7D82078002819D003F0F5
:10AB700089FB0146E01CFDF737FC104A01261460F2
:10AB8000E979AB7920780902194381420BD90C4944
:10AB900090800978491E084206D10A4901200870B0
:10ABA00002E0002602E09180FFF748FD304670BDCC
:10ABB0007CF5FF1F943F010038F4FF1F74F5FF1F61
:10ABC000713F010064F5FF1F10B5154A1549507813
:10ABD00009780024884220D1507911790002084375
:10ABE00007281AD1114B10481860417A007A0902DF
:10ABF0000143D0799279000201241043884209D997
:10AC00000B4899800078401E014204D10949012077
:10AC1000087000E09880FFF711FD204610BD00008D
:10AC20007CF5FF1F953F0100E8F2FF1F74F5FF1F41
:10AC3000713F010064F5FF1F074800214170C160AA
:10AC400001614161418081808161C161C180018177
:10AC5000016241817047000084F5FF1FF8B54A4E3C
:10AC6000B0887188494F00257C1C884218D3B06990
:10AC7000002815D17561B580012339787A1C1846F2
:10AC800007F0BAF970807088002809D040487761D1
:10AC90000078012801D8746102E07088401C70803F
:10ACA000708800283AD1F068002801D0F56035E0BE
:10ACB0003069002832D03649097801290ED83D7014
:10ACC000B58002237A1C0021012007F095F97080DD
:10ACD0007088002800D0746135611FE03C7801273E
:10ACE000202C00D300243946A14001421AD0601C18
:10ACF000C1B2264A02231170B5800120521C07F010
:10AD00007BF970807088002804D0204870617088BA
:10AD1000401C70803069A740B843306170880028BB
:10AD200006D102E0641CE4B2DAE7B069002828D05A
:10AD30007088B188174F401A84B23878410016489D
:10AD4000405AA04200D2044614480078002805D09A
:10AD5000802108432246716901F05EFD7069104947
:10AD600000197061B088001980B2B08009888842EB
:10AD700008D2387841000848405AA04202D1012048
:10AD8000B061F8BDB561F8BD84F5FF1FB0130020B8
:10AD90007C3F010063F5FF1F783F0100723F010017
:10ADA0007E3F0100F8B51C4C002620891B4D1C4F2E
:10ADB000002803D1E5613888E0802681E088218978
:10ADC000421A1848E169007801F0B6F8E16980B2EA
:10ADD0000918E161218909188BB22381002809D063
:10ADE00039888B4206D21049104A09784900515AD5
:10ADF000814210D90E48017801200129009003D822
:10AE00000021064A022003E029786A1C02205B1E0A
:10AE100007F08CF92681F8BD84F5FF1FF11300209F
:10AE2000803F0100733F010063F5FF1F783F010081
:10AE30007D3F010010B50446000702D52046FFF70C
:10AE40000DFF600702D52046FFF7ACFF10BD0000E4
:10AE5000034804498078085C034908700120704762
:10AE60007CF5FF1F82F4FF1F7013002010B507F060
:10AE7000C1F802490870012010BD000070130020C5
:10AE800010B50B490022C878012804D0022804D04C
:10AE9000032806D103E0074A02E0002010BD064A5D
:10AEA000521C8978002307F0A7F8012010BD00008C
:10AEB0007CF5FF1FB013002083F4FF1FFEB544484C
:10AEC000007800287ED0434E002031788446481C0C
:10AED00030704148042300784200821893405B1E82
:10AEE0000192994203DB0021317001218C463B4ADB
:10AEF00000251188FF2901D2491C118041003848E2
:10AF0000405A364900900988884200D101253549C8
:10AF1000002009788E4648E000216246002A0DD0C4
:10AF2000314A135CFF2B01D25B1C13542F4B1B5C6B
:10AF3000002B03D0125C9A4200D301212B4A02233A
:10AF4000145C019A934022469A40009B9A4203DA8D
:10AF5000002C01D0012200E00022002D06D0002AA2
:10AF600004D00123376983403B433361204B1B5C92
:10AF70009C420CD01C4C245C9C4206D301243769B3
:10AF800084403C43346100243470184C235400291D
:10AF900009D0002A04D10121326981401143316175
:10AFA000114A00211154401CC0B27045B4D3002D89
:10AFB00002D00A49002008803069002806D0708835
:10AFC000002800E002E001D1FFF748FEFEBD0000CE
:10AFD00061F5FF1F84F5FF1F63F5FF1F7EF4FF1F60
:10AFE000743F01007C3F010080F4FF1F81F4FF1FCC
:10AFF00082F4FF1F0A480A498078C978002802D0E5
:10B00000084A815409E0094B0020074A1B7802E0F6
:10B010001154401CC0B29842FAD30120704700007E
:10B020007CF5FF1F81F4FF1F82F4FF1F7C3F0100AE
:10B0300010B50348807807F077F8012010BD0000B4
:10B040007CF5FF1F38B50D490022C878012804D0CF
:10B05000022804D0032806D103E0002038BD084AA6
:10B0600000E0084A521C00230093CB798C791B0224
:10B070002343897807F05AF8012038BD7CF5FF1F7B
:10B08000F113002083F4FF1FF8B5EFF31080C00721
:10B09000C00F72B6564D0021EC68E9602A78009224
:10B0A0002970002800D162B6E00708D001F0DCFA70
:10B0B00007F0EAF84F480068002800D08047E00613
:10B0C00006D501F09FFB4C480068002800D080475F
:10B0D000A00606D501F04AFB48480068002800D0C9
:10B0E0008047600704D546480068002800D08047A4
:10B0F000022C09D143480168002902D04248007A55
:10B1000088474148FF210172200767D53F4FEFF381
:10B110001080C207D20F72B6A9686868884257D1FA
:10B12000012156E0EFF31081CE07F60F72B63849D1
:10B130000C5C1921401CFDF789FA6960002E00D1D2
:10B1400062B620462207D30F21066207090FD20FED
:10B15000002908D15C00A418E4003C5D0026A40688
:10B16000240F0D2C0AD08C005B00E3189A18D6002F
:10B17000BA5D9206120F012A13D01DE02869022140
:10B1800088432861387E4006400E3876387C400679
:10B19000400E38741F486E7001680029B7D0022035
:10B1A00014E0002902D1C007C00F68701948015986
:10B1B000002901D004208847B85D8006000F0928C7
:10B1C000A5D1144801590029A1D0082088479EE73D
:10B1D0000021002A00D162B60029A3D000980028DF
:10B1E00004D00949087DDF2210400875F8BD000031
:10B1F00088F4FF1FA03F0100A43F0100A83F010009
:10B20000AC3F0100B03F0100802007400016002045
:10B21000C01C0020B43F010010B51D48402404703C
:10B220001C4841680522120411434160416B22030E
:10B2300011434163182001F051FB1748017B802224
:10B2400011430173017B0906FCD41449124B090A0E
:10B25000803B197711490A0C0F4960390A740F4A6B
:10B26000120E0A75FF2119700D490968002900D0D6
:10B2700004210C4A1268002A00D00222114319222C
:10B28000114319710470017B2143017310BD00004B
:10B290009CF4FF1F0080044000210740001600209E
:10B2A000AC3F0100B03F010070B500F019F9002873
:10B2B0002AD01648022404704470154E03203463CB
:10B2C000307014480546FDF7A8F9022808D911493D
:10B2D00020461F39FDF7B2F929462046FDF7AEF9A1
:10B2E0000D488021007822460843084901F094FA6D
:10B2F0002846FDF792F9316B401A2946FDF79EF971
:10B30000044901200839087370BD00003214002080
:10B31000A8F5FF1FBB240020823F010010B5104993
:10B320000878022808D003280FD0042810D0052858
:10B3300001D10020087010BD0A48C07B282801D028
:10B34000A828F8D100F06CFA10BD00F077FD10BD10
:10B35000054880210078084300F08AFDF5E70000E9
:10B36000A8F5FF1F94240020823F010010B51D4A5C
:10B37000117800290FD0012910D01B480529007829
:10B380001BD0072927D000F073FD1849022008734D
:10B3900000F054FD10BD00F00FF910BD13481F3828
:10B3A000C07B2A2803D02F2804D0AA28F5D100F08A
:10B3B00015FB10BD00F0A2FA10BD012181400C4820
:10B3C0000068014201D0012000E00020094A0AA1E2
:10B3D00001F0D2FA10BD00201070106B1F28DAD0D7
:10B3E00010BD0000A8F5FF1F833F0100B32400201B
:10B3F0006CF5FF1F3F0400002E2E5C2E2E5C2E2EBF
:10B400005C736F757263655C7573625C6D73635CAE
:10B41000757362645F6D73632E63000010B5144C26
:10B420006068E060002801D0012010BD1148FDF7E0
:10B43000F4F8002814D00F480838007B000604D523
:10B440000D4880210078084308E00A481F30FDF7C6
:10B45000E4F8216B884203D00848007800F008FD2A
:10B46000044901201731087300F0E8FC002010BDEA
:10B47000A8F5FF1F9C240020823F0100833F0100AC
:10B4800010B5124801798F200140080605D508073C
:10B49000000F01221204824001E001228A400C4880
:10B4A0000478802004438C420ED10A480068104280
:10B4B0000AD00948FDF7B1F80849884204D10D22A5
:10B4C0000549204601F0A8F910BD00007CF5FF1FDA
:10B4D000823F01006CF5FF1FB324002055534253F7
:10B4E00070B50C48FDF799F80A4C0225173400286E
:10B4F00008D020461F38007B000608D40648007894
:10B5000000F0B6FC257300F099FC002070BD01200E
:10B5100070BD00009C240020833F010070B51148DD
:10B52000FDF77BF8104C216B884202D82063032082
:10B5300000E0042020700D4880210078226B084331
:10B540000B4901F069F907481F300546FDF765F81A
:10B55000216B401A2946FDF771F802490020173186
:10B56000087370BD9C240020A8F5FF1F823F0100D6
:10B570003214002010B506480649028806480078B3
:10B5800000F0DAFC05490863FFF7F0FE10BD00008B
:10B59000883F010032140020833F0100A8F5FF1FFF
:10B5A00010B50446400702D50020FFF7E3FF20074F
:10B5B00001D5FFF7B3FE10BDF8B5704E316B1F29F2
:10B5C00001D20A4600E01F2200206D4D6D4B02E0C3
:10B5D0001C5C2C54401C9042FAD36B4880220078AB
:10B5E0000127104300901F2970D16548FDF715F819
:10B5F000664988426AD1281DFDF70FF8604C1F3458
:10B60000211DFDF71BF820461738FDF706F82146E7
:10B610000831FDF713F8687B002804D1A87B0028C7
:10B6200001D0102801D9277374E0E87B2A283BD089
:10B6300020DC1A2847D00EDC0428F4D006DC0028D1
:10B640003BD00328EFD100F075FBF8BD1228EAD1FA
:10B6500000F0AAF8F8BD23283CD006DC1B282FD028
:10B660001E28E0D100F0CCF8F8BD252835D02828D8
:10B67000D9D13BE09E2836D00EDC5528D3D004DC4F
:10B680002F2842D03528CED103E05A281FD0912848
:10B69000C9D100F01DFCF8BDA12821D0A3284ED0AF
:10B6A000A82823D0AA28BED100F084FA0028F2D01E
:10B6B000287B00063BD43770F8BD00F013FCF8BDC2
:10B6C00000F0ECFBF8BD00F047FAF8BD3BE000F0FD
:10B6D00011FAFAE700F0F2FAF7E700F0C9FAF4E736
:10B6E000FFF7E2FDF1E700F07DFBEEE700F062FA24
:10B6F0000028EAD0287B000604D50220307000F034
:10B700008FF8E2E72248007815E0287C800704D40F
:10B710000020207300F092FBD7E700F04BFA0028DE
:10B72000D3D0287B000602D437703762CDE71648A5
:10B7300080210078084300F09BFB0220E9E7009895
:10B7400000F096FB6FE7104C009800F091FB20781A
:10B75000104C0107090F01200004884021680C4D9E
:10B7600008432060287800F083FB28788740206811
:10B770000743062027603070A7E70000A8F5FF1FE9
:10B780009424002032140020823F0100555342438C
:10B79000833F010070F5FF1F02490020087001205F
:10B7A000704700007013002010B5FFF799FE0028C5
:10B7B0001FD0104B00201870802159700221997001
:10B7C000D97020241C7158719871D8710A48016889
:10B7D00008200A78002A02D01A54491C00E01C54A0
:10B7E000401CC0B22428F4D3044924200863FFF786
:10B7F00095FE10BD3214002034F4FF1FA8F5FF1F82
:10B8000010B50548C07CC107044800D00121017370
:10B8100000F014FB10BD000094240020B32400208D
:10B82000F8B5314D314FA969686A002688420AD3BC
:10B83000387880210024084300F01AFB2C48067356
:10B8400000F0FCFA08E02B48007841002A48445AEE
:10B85000E86A844200D30446FFF7E0FD002800D1E7
:10B860000024A86A00282DD0002C0ED0A96AE8690F
:10B870008022411838781043224600F0CDFFA86A94
:10B880000019A862E86A001BE86229696869AA6A67
:10B890004143914203D1AE62696A08186862144854
:10B8A00008300746FCF7B9FE001B3946FCF7C6FE18
:10B8B000002C06D0E86A002803D1032028700C4829
:10B8C0000673F8BD002CE0D02969E86A4018401ED4
:10B8D000FCF7BCFE69690246884200D90A46E9695C
:10B8E000686A06F091FCC1E7A8F5FF1F823F0100DE
:10B8F000B324002063F5FF1F843F0100F8B5334CEB
:10B900000025A169606A884208D331482563007820
:10B9100000F0AEFA2F48057300F090FAFFF77EFDB5
:10B92000002806D0206B002824D0A06A002802D06E
:10B9300010E025631EE02169E06A4018401EFCF714
:10B9400085FE61690246884200D90A46E169606A5B
:10B9500006F05AFC00202049A76A266B08E0E3693C
:10B960003A189A5C0B5C9A4201D0256202E0401CB6
:10B97000B042F4D3266BA06A8119A162E06A871BEA
:10B98000E7622269606942438A4203D1A562616A23
:10B99000081860620F4808300546FCF73EFE801B21
:10B9A0002946FCF74BFE002E0CD0002F02D0207849
:10B9B000052807D1206A002805D000200549087312
:10B9C00000F03CFAF8BD0120F8E70000A8F5FF1FE1
:10B9D000833F0100B324002032140020F8B5384D15
:10B9E000384FA969686A0026884207D336482E6313
:10B9F000007800F03DFA3E7300F020FAFFF70EFDEC
:10BA0000002800D12E63296BA86A40182969884252
:10BA100005D9FE222DA1002000F0AEFFF8BD0020C8
:10BA2000334905E0AB6A0A5C1B18EC69401CE25420
:10BA30002A6B9042F6D3A86A8018A862E96A891A2C
:10BA4000E962002A25D0002914D1002812D02969E2
:10BA50004018401EFCF7FAFD69690446884200D987
:10BA60000C462246E969686A06F0E6FBAE62686A3F
:10BA700000190DE069692B690A465943814208D1D2
:10BA8000E969686A06F0D8FBAE626969686A4018BD
:10BA900068620C4808300090FCF7BFFD2C6B0099E1
:10BAA000001BFCF7CBFD002CB8D0E86A002802D0C0
:10BAB00028780528B2D13E7300F0C0F9F8BD000027
:10BAC000A8F5FF1FB3240020833F01002E2E5C2E1B
:10BAD0002E5C2E2E5C736F757263655C7573625C91
:10BAE0006D73635C757362645F6D73632E630000D6
:10BAF0003214002070B5FFF7F3FC002824D0FFF7C4
:10BB00008DFC002820D011480021017006224270CF
:10BB10000F4B81701A7A0824D201C27001714171F1
:10BB20008171C1710B481C630546FCF776FD08283E
:10BB300008D9084920461F39FCF780FD29462046D0
:10BB4000FCF77CFDFFF7EAFC70BD0000321400201A
:10BB5000A8F5FF1FBB24002070B5FFF7C1FC00282B
:10BB600020D0FFF75BFC00281CD00F480321017098
:10BB700000210E4B41701A7A0424D2018270C170E8
:10BB80000B481C630546FCF748FD042808D9084902
:10BB900020461F39FCF752FD29462046FCF74EFD92
:10BBA000FFF7BCFC70BD000032140020A8F5FF1F99
:10BBB000BB240020F8B52A48FCF72FFD284D00BA19
:10BBC000040A113D287D24020443264E002074629D
:10BBD000B062E87B2F280AD004DC28280BD02A2862
:10BBE0001CD104E0A82810D0AA2817D109E0FFF73B
:10BBF00015FC002830D0E87DA97D0002084344BA36
:10BC00000CE0FFF70BFC002826D01548001DFCF7C0
:10BC100004FD00BA040A287E240204433069444328
:10BC20000F48F4620938FCF7F8FC0D4F01260E3777
:10BC300000280DD0A04210D0287B000604D50A4869
:10BC400080210078084301E00848007800F010F9EE
:10BC50003E7300F0F3F80020F8BD0120F8BD0000AD
:10BC6000A5240020A8F5FF1F823F0100833F0100AB
:10BC700010B5FFF735FC00281AD0FFF7CFFB0028DE
:10BC800016D00C4A0C489169491E0B0E03700B0C20
:10BC900043700B0A8370C17011690B0E03710B0C9A
:10BCA00043710B0A8371C17108201063FFF736FCE2
:10BCB00010BD0000A8F5FF1F3214002070B5FFF77B
:10BCC0000FFC00282ED0FFF7A9FB00282AD0164829
:10BCD00000210170417081700821144AC17091697E
:10BCE0000C240B0E03710B0C43710B0A8371C17191
:10BCF0000221017211690B0C43720B0A8372C1722B
:10BD00000B4814630546FCF788FC0C2808D9084941
:10BD100020461F39FCF792FC29462046FCF78EFC92
:10BD2000FFF7FCFB70BD000032140020A8F5FF1FD8
:10BD3000BB24002070B5FFF7D3FB00282ED01B4892
:10BD40007021017000211A4B41705A68DD68144659
:10BD5000AC4306D006248470282404734173DA604F
:10BD60000AE0002A1BD0134A127B002A1BD00522AE
:10BD70008270202202734173C1700171417181711F
:10BD80000A22C271017241728172C1728173C173E0
:10BD90000174417412201863FFF7C0FB70BD0222CA
:10BDA00082703A22E6E781700173E4E732140020E2
:10BDB000A8F5FF1FB324002010B505490020086036
:10BDC0000449FCF73BFC044907200870012010BD22
:10BDD00070F5FF1FB3240020A8F5FF1F10B5FFF773
:10BDE000EBFF10BD70B5FFF77BFB00281DD00F489F
:10BDF0002022027000214170C1770D4C0320226384
:10BE000020700C48802100780843084900F004FDA8
:10BE100009480546FCF701FC216B401A2946FCF74E
:10BE20000DFC054901200839087370BD321400204B
:10BE3000A8F5FF1F823F0100BB24002010B5084970
:10BE40000848FCF7FBFB0848802100780D220843D6
:10BE5000034900F0E1FC05490520087010BD000011
:10BE6000B324002055534253823F0100A8F5FF1F21
:10BE700010B5044600F092FC200605D52107090FF5
:10BE800001200004884001E00120A04002490A6826
:10BE90001043086010BD00006CF5FF1F10B50A4884
:10BEA000817C04461F34002904D001202073FFF751
:10BEB000C5FF10BDC07C0549C007C00F486006F033
:10BEC000B9F90020F2E7000094240020A8F5FF1F34
:10BED00010B5034900200873FFF7B0FF10BD000044
:10BEE000B324002010B51048FCF797FB0E4C173414
:10BEF00000280FD020461F38007B000604D50B48D1
:10BF000080210078084301E009480078FFF7B0FF7E
:10BF1000012004E0FFF782FA002803D000202073FC
:10BF2000FFF78CFF10BD00009C240020823F010021
:10BF3000833F010070470000F7B5074682B000203C
:10BF400000903807860E3348F50028180190448881
:10BF5000002F15D130484078002809D07008012101
:10BF600081402D48103003F016F8002005B0F0BDD8
:10BF70002848405D8006000F0D2801D10120009067
:10BF80000498A04206D2FF22EE3224A1002000F045
:10BF9000F3FC049C1F4A0020B101C032891803E061
:10BFA000039A0B5C1354401CA042F9D31A48143076
:10BFB000C15D0198174F4180174876080069795D87
:10BFC000F040C0074906C00FC90F88420FD103983F
:10BFD000C1798279080200991043002901D0002814
:10BFE0000CD001210C48B140103002F0D4FF0A48B7
:10BFF0000069F040C00708D0C82007E006480121CA
:10C00000C943103002F0AFFFF1E788207855204691
:10C01000ACE700000016002088F4FF1F2E2E5C2ED7
:10C020002E5C2E2E5C736F757263655C6869635F4E
:10C0300068616C5C667265657363616C655C757381
:10C0400062645F6B696E657469732E630000000043
:10C0500010B5FFF715FA10BDFEB5574A574D1078C9
:10C06000574CC006C00E02D001287CD18CE0554947
:10C07000D0780B785149544E544FC978062810D0C7
:10C0800006DC012809D0022815D003286BD14FE027
:10C09000072832D00F2866D166E04D482060122074
:10C0A00070E0002B5FD0002903D04A4820600A20AE
:10C0B00068E04948FAE7002B01D1012979D0022034
:10C0C000002904D000977870002092780DE0009647
:10C0D0007070F9E700990B78002B05D0CB788E783B
:10C0E0001B02334359180091401C8242F2D1009840
:10C0F000017800295DD0206040E0002B59D0072056
:10C10000002904D000967070002092780DE000970E
:10C110007870F9E700990B78002B05D0CB788E78F2
:10C120001B02334359180091401C8242F2D1DEE7D2
:10C130002A4800909078032801D0002009E002F0FE
:10C14000FFF80DE000990B78002B01D059180091F1
:10C15000401C91788142F5D100980178002928D0BF
:10C16000206000780EE024E01D48007800281FD0F1
:10C170001C4800902060017800291AD0C17882788C
:10C1800008021043019005E001A9684600F02EF86E
:10C1900000280DD0A1880198814208D980B21249A7
:10C1A000A0800978491E084201D101202871012090
:10C1B000FEBD0020FEBD00007CF5FF1F60F5FF1FE7
:10C1C00074F5FF1F6F3F0100A8120020DFF2FF1F70
:10C1D0002440010037400100364001007240010058
:10C1E000703F010038400100713F010070B51A4AEC
:10C1F0001A4CD3781A4A25781478174A194E1279AE
:10C20000212B02D0222B24D118E0AA4201D0A24235
:10C210001FD1154A1378154A002B127801D1012A33
:10C2200017D0002A08D0124A02601046114A12881C
:10C2300080183060092009E00F4AF5E7AA4201D0D2
:10C24000A24206D10D4830600D48008808600120E8
:10C2500070BD002070BD00007CF5FF1FE0F2FF1FE5
:10C26000E2F2FF1F74F5FF1F6F3F010063F5FF1F30
:10C27000DFF2FF1FE6F2FF1FA812002000400100BE
:10C280002240010070B51D481D4B0078C106C90E43
:10C290000AD01D461948143D1A4C6A7800790129C4
:10C2A00006D0022928D10AE015480E38186021E08E
:10C2B000002A21D0A97888421ED2002016E08F21C2
:10C2C0000840010605D50607360F01210904B140D3
:10C2D00001E001218140002A01D100070CD1A868AA
:10C2E000084209D0E868084000D001202070000A08
:10C2F00060701C60012070BD002070BD7CF5FF1FC8
:10C3000074F5FF1F7013002070B5274B0246187894
:10C310001946C0064988254EC00E04D001282BD0EE
:10C32000022829D111E0012926D10224002A05D0B2
:10C33000012000F06FFAF088204304E0002000F0B4
:10C3400069FAF088A043F0802CE01C798F2004402B
:10C35000200605D52007000F01252D04854001E0AA
:10C360000125A5407078002806D0200704D0B068C9
:10C37000284201D0002901D0002070BD002A05D03C
:10C38000204600F00BFAF06828430AE030692842A2
:10C3900008D12046FEF718F92046FFF759FEF0684D
:10C3A000A843F060012070BD7CF5FF1F60F5FF1F02
:10C3B000F8B55A4800260178C906C90E7ED1574FF4
:10C3C00080781C3F00287AD0554801783846C078DC
:10C3D000002901D1012871D0002801D0514C70E012
:10C3E000514C6EE06078022805D0042847D005281B
:10C3F00047D0072860D1494861798078814239D196
:10C4000078702079B8704A490020484A0B8802E0C9
:10C4100000211154401C9842FAD301250120B9682B
:10C42000A840084202D02846FEF738F9012000044F
:10C43000B968A840084204D0284680210843FEF786
:10C440002DF96D1C102DE9D33A48B8600020F86032
:10C4500038613D460120FEF7D5F8E079400604D565
:10C46000E98801200143E98026E0E888400840008F
:10C47000E88021E0E078A178000208431DE0E6783A
:10C480001AE0002E18D1A5788F200540280605D582
:10C490002907090F01200004884001E00120A8407D
:10C4A000B96801432046B960FEF79CF82846FEF7BC
:10C4B00007F9284600F022F9207801E02AE004E09C
:10C4C0000419207800288DD11FE0002501247D70FB
:10C4D00080260120B968A040084202D02046FEF71D
:10C4E000DDF801200004B968A040084203D02046CE
:10C4F0003043FEF7D3F8641C102CEAD3FD600D48DE
:10C500003D61B8600020FEF77DF8044879788078B6
:10C51000884201D00020F8BD0120F8BD7CF5FF1F46
:10C520006F3F0100DFF2FF1FA812002077F4FF1F0A
:10C53000E4F2FF1F01000100F0B585B00027454877
:10C540000397019700783E46C006C00E01287ED1B1
:10C5500040491C394878002876D0002002903E4897
:10C5600002780846C078002A01D101286FD000283F
:10C5700001D03A4C64E03A4C62E06078022805D081
:10C5800004280ED005281ED0072857D131486179DC
:10C590001C384078814251D0E078A17800020843ED
:10C5A0004DE0A778E678002001902A480179B94249
:10C5B00044D18078B04241D1012002902948C15D28
:10C5C0000391C6553AE023490879B84236D1A0789C
:10C5D0008F22104000900006009804D50007000F3D
:10C5E00001252D0400E0012585408878B04214D152
:10C5F00018481C38816829438160C168A943C1601B
:10C600002046FDF7EFFF0098FEF75AF8009800F07B
:10C6100075F801982843019010E0039886420DD1E7
:10C62000019828420AD10B481C388168A9438160CF
:10C63000C168A943C1600098FEF730F8207804195A
:10C640002078002899D1029805B0F0BDFFE70020BE
:10C65000FAE700007CF5FF1F6F3F0100DFF2FF1FCC
:10C66000A812002077F4FF1F70B501201C490006B6
:10C670000860BFF34F8FBFF36F8F0120194D002467
:10C68000810049190C70401C1028F9D31921164853
:10C69000FBF7C1FF1548164944608460C46004700C
:10C6A000447040224A800A46C0324A60C8220A705A
:10C6B0000C72104ACC614A610D2129700E4901614A
:10C6C00008484038017D022211430175FF210170A5
:10C6D000017201730476182000F000F970BD0000AB
:10C6E00080E100E0C0200740C01C002088F4FF1F4C
:10C6F000001600204017002055555555F8B5054641
:10C70000154F2C073E4600060121C03E240F00288D
:10C710000EDA6000401C8140104802F030FC20021C
:10C72000C11960018019803141610021C161F8BDEA
:10C7300068008140C943094802F015FC07486101BF
:10C74000001D425D881942802202D219426088226F
:10C75000725400210172F8BDC016002098F4FF1F2A
:10C7600010B5FDF7A1FEFFF739FB10BD02480179B6
:10C77000DF221140017170478020074010B5FEF79D
:10C780009DFBFDF795FE10BD002903D1400602492F
:10C79000400E087670470000802007400007810E99
:10C7A0000348081801780222114301707047000005
:10C7B000C020074010B5082202490020FFF7BCFB4B
:10C7C00010BD00007CF5FF1F10B503480121490290
:10C7D000C06802F019F910BD4CF0FF1F10B500221F
:10C7E0001146802000F018F810BD000010B5034875
:10C7F000034902780020FFF79FFB10BD713F010045
:10C800007013002002480179202211430171704702
:10C810008020074070470000F8B50007114F840ED4
:10C820001646A41CE200D01946803D460023A00114
:10C83000C035451902E0C85CE8545B1CB342FAD32A
:10C84000094960080969C140C90701D0882100E091
:10C85000C821B954012181400348103002F09BFBEC
:10C860003046F8BD0016002088F4FF1F00207047F6
:10C8700030B47446641E2578641CAB4200D21D4659
:10C88000635D5B00E31830BC18470000002805DB3F
:10C89000C106C90E012088400149086070470000A8
:10C8A00080E200E0002809DBC106C90E01208840B3
:10C8B00003490860BFF34F8FBFF36F8F70470000CD
:10C8C00080E100E0002805DBC106C90E0120884098
:10C8D000014908607047000000E100E0002805DB26
:10C8E000C106C90E01208840014908607047000058
:10C8F00000E100E010B5002A06DA52005208D21D0D
:10C90000D308DB00102203E0D21C93089B000C220A
:10C91000002B02D09C188C4201D9012010BD821836
:10C920008360411802604160C91AD018884202D859
:10C9300010600246F9E70020106010BDB0B5044653
:10C9400003F05CFA002804D0034F0249BC4620687B
:10C9500000DFB0BDFFFF0000BDF80000B0B5044629
:10C9600003F04CFA002803D0024F2068BC4600DFD9
:10C97000B0BD000015F80000F8B516460F460028B7
:10C980001BD1EFF31080C507ED0F72B600231A46D6
:10C990001946184600F02AFA040003D131463846F9
:10C9A00000F07CFA002D00D162B6002C05D1EFF327
:10C9B0000380C00601D105F06DFFF8BD704700008F
:10C9C00010B528220D490E48FBF782FC06F020F82E
:10C9D0000C4806F017F805F03FFE0B4901220860ED
:10C9E0000A4952020A600A4A012111600949400AB3
:10C9F00008600A490848086010BD00009031010035
:10CA00009C02002011D50000DCF5FF1FB8F5FF1FC8
:10CA1000BCF5FF1FC0F5FF1F9C000020C4F5FF1FE1
:10CA200000B591B0FDF778FB402801D9402001E026
:10CA300000280DD081B2684604F01CFF010007D029
:10CA40006846FDF791FB002802D0012001F0F4FDBB
:10CA500004F094FF0146402801D9402101E000295B
:10CA60000DD06846FDF764FB002808D081B2684607
:10CA700004F064FF002802D0012001F0DDFD01F088
:10CA8000F3FD11B000BD0000044841788078814278
:10CA900001D001207047002070470000FCF0FF1F0C
:10CAA00030B50546EFF31080C407E40F72B6284690
:10CAB00000F007F8A968081A401E002C00D162B6E1
:10CAC00030BDEFF31081CB07DB0F72B606C8083814
:10CAD0008A4201D3501A02E080681018401A002BD5
:10CAE00000D162B67047EFF31083DB07DB0F72B63D
:10CAF0008260C160002101604160002B00D162B6FC
:10CB00007047000070B50446EFF31080C507ED0FC5
:10CB100072B603CC083C884201D0012000E000201E
:10CB200042220DA1FFF728FFE16820680E5C401C3F
:10CB30002060A16888420AD3884201D1012000E028
:10CB40000020472204A1FFF717FF00202060002DDE
:10CB500000D162B6304670BD2E2E5C2E2E5C2E2E7D
:10CB60005C736F757263655C6461706C696E6B5C3D
:10CB7000636972635F6275662E63000070B5044678
:10CB8000EFF31080C507ED0F72B66268E06881545C
:10CB90006068401C6060A16888420AD3884201D165
:10CBA000012000E00020302209A1FFF7E5FE00206F
:10CBB000606003CC884201D0012000E000203522D3
:10CBC00003A1FFF7D9FE002D00D162B670BD0000B1
:10CBD0002E2E5C2E2E5C2E2E5C736F757263655C40
:10CBE0006461706C696E6B5C636972635F627566C9
:10CBF0002E630000F8B514460E460746FFF761FFA6
:10CC0000844200D220460546002404E03846FFF75F
:10CC100079FF3055641CAC42F8D32846F8BDF8B50E
:10CC200014460E460746FFF73BFF844200D22046DB
:10CC30000546002404E0315D3846FFF79FFF641C81
:10CC4000AC42F8D32846F8BD10B50C48C078012195
:10CC5000C00948402A220AA1FFF78EFE1449012488
:10CC60006402084622461038FFF73DFF114922466C
:10CC700008461038FFF737FF10BD000000B006402F
:10CC80002E2E5C2E2E5C2E2E5C736F757263655C8F
:10CC90006869635F68616C5C667265657363616C2B
:10CCA000655C6B6C32367A5C756172742E63000061
:10CCB000980E0020A810002010B500F083FD10BDD4
:10CCC00010B500F07FFD10BD02488079002800D02B
:10CCD000012070471C2300200248C079002800D0A2
:10CCE000012070471C2300200248007A002800D051
:10CCF000012070471C230020F8B58D212648FBF742
:10CD000088FC8D272548FBF788FC234C244E234DB7
:10CD10004034B04213D168792A79010211438D2938
:10CD200001D20A4600E08D228D2901D90F4600E08C
:10CD30008D271A491848FBF7BBFB0020E0718D21B5
:10CD40001648FBF766FC15493046FBF777FC2F7158
:10CD5000390A697110494122C91DE81DFBF7A8FB7A
:10CD6000607A227A01020D48114340300172090AAB
:10CD70004172A17A8172E17AC1728A0006490C304F
:10CD80004C31FBF795FB04488030017B0348803031
:10CD9000017300F0BBF8F8BD8C220020002F0020AA
:10CDA000646C766B10B5094CE17A102901D3002030
:10CDB00010BD064A8900403A89184C31FBF73EFC09
:10CDC000E07A401CC0B2E07210BD0000402F00208D
:10CDD00010B541210448FBF71CFC03480021393001
:10CDE00001724172C17210BD072F0020FFB581B0E2
:10CDF0001D4616460F461A48FBF7D4FA441C019804
:10CE0000002802D03946FBF704FC0020002E00D099
:10CE10003080002D00D028701149C91FC879002822
:10CE20001BD0BC4201D8224602E0E01B41183A4622
:10CE30000B4C0198C91D3934002804D0607A237A3C
:10CE4000000218433080002E02D00198FBF730FB1F
:10CE5000002D01D0A07A2870012005B0F0BD00009F
:10CE6000072F00200148007B70470000802F002022
:10CE70000549CA7A002A04D00A460C320260C87AF0
:10CE80007047002070470000402F00200248807942
:10CE9000002800D001207047002F0020F3B581B09A
:10CEA0000746FBF77FFA124D441C41263146E81D28
:10CEB000FBF7AFFB412C02D83946224602E0413C49
:10CEC000E1193246E81DFBF7F3FA094C02984034A9
:10CED0002072000A607200F084F9002801D001205D
:10CEE00004E000F080F9002800D00220A072FEBD0E
:10CEF000002F00200149087370470000802F002098
:10CF00000149887170470000002F002070B5002291
:10CF100011461046FCF708FC092220492048FBF77F
:10CF2000C7FA204C22781046627812021043A27889
:10CF3000E1781204104309061B4D0843A8420FD1A3
:10CF40006079217900020843092804D260792179A7
:10CF500002020A4300E0092212491148FBF7A8FA2D
:10CF60000F492846FBF76AFB0D4909208880207885
:10CF70000146607800020143A07800040143E07894
:10CF800000060143A94205D16079217900020843D6
:10CF9000092802D2024801F00DFF70BDF0410100E6
:10CFA0001C23002000FC0100646C766B10B5034963
:10CFB0008871084601F0FEFE10BD00001C23002011
:10CFC00010B50349C871084601F0F4FE10BD000019
:10CFD0001C23002010B503490872084601F0EAFE40
:10CFE00010BD00001C23002070B506460F484024E9
:10CFF00045080F486D0041084900A9420CD94C1B57
:10D00000402C01D8012000E000200A4A0AA1FFF7C5
:10D01000B3FC402C00D94024224629463046FBF779
:10D0200047FA1248761C466070BD000011D7000018
:10D0300025D700001C0800002E2E5C2E2E5C2E2E04
:10D040005C736F757263655C6869635F68616C5C73
:10D05000667265657363616C655C6961705C66735B
:10D060006C5F666C6173682E63000000D0F2FF1F76
:10D0700070B506460F48402445080F486D0041082A
:10D080004900A9420CD94C1B402C01D8012000E0DA
:10D0900000200A4A0A49FFF76FFC402C00D94024BF
:10D0A000224629463046FBF703FA0648761C0660FE
:10D0B00070BD0000E5DF0000F1DF00008E0700001A
:10D0C00038D00000D0F2FF1FF8B50024E4430F462B
:10D0D0000646002512E0705D082102F075F9000691
:10D0E00044400A490820002C02DA64004C4000E069
:10D0F0006400401E0006000EF5D16D1CBD42EADB47
:10D100002021204602F060F9C043F8BDB71DC104DC
:10D11000F8B50E4617462021C04302F055F90446E3
:10D12000002512E0705D082102F04EF9000644402F
:10D130000A490820002C02DA64004C4000E0640038
:10D14000401E0006000EF5D16D1CBD42EADB202119
:10D15000204602F039F9C043F8BD0000B71DC104F4
:10D1600070B514460D460646FF2A07D8FF22DE3268
:10D170000AA10020FFF700FC022070BD00F06EFD48
:10D18000002801D0102070BD2A462146304600F00C
:10D190001DFF0028F7D01F2070BD00002E2E5C2E32
:10D1A0002E5C2E2E5C736F757263655C6461706CAF
:10D1B000696E6B5C647261672D6E2D64726F705C5A
:10D1C0006961705F666C6173685F696E74662E6317
:10D1D00000000000C1060007000F002900DB093035
:10D1E0007047002070470120704710B500231A4691
:10D1F00000F022FB002800D0012010BD10B505F082
:10D2000031F9012800D0002010BD0000F8B5164EFD
:10D21000012530780024ED03012806D0FF223832A2
:10D2200012A10020FFF7A8FB0AE0B078022700282F
:10D2300008D0FF223E320DA10020FFF79DFB377082
:10D240000220F8BD204600F02DF8002802D03770EB
:10D250002120F8BD012080022418AC42F2D3012025
:10D26000B0700020F8BD0000D8F0FF1F2E2E5C2EFD
:10D270002E5C2E2E5C736F757263655C6461706CDE
:10D28000696E6B5C647261672D6E2D64726F705C89
:10D290006961705F666C6173685F696E74662E6346
:10D2A00000000000F8B5254E05463078012805D06D
:10D2B000FF2223A10020FFF75FFB1AE00127BF0236
:10D2C00039462846FBF7C2F90224002902D0FF2282
:10D2D000083209E0F07800280DD0F168B0684018F5
:10D2E000A84208D0FF220F3215A10020FFF744FB0F
:10D2F00034700220F8BD01227F20D2038002012178
:10D30000954203D3854201D2002000E00846002860
:10D3100010D0F170F7602846B56001F025F9252896
:10D3200003D00028E6D03470F8BD284600F096FC03
:10D330000028F9D034702020F8BD0000D8F0FF1F7D
:10D340002E2E5C2E2E5C2E2E5C736F757263655CC8
:10D350006461706C696E6B5C647261672D6E2D64C4
:10D36000726F705C6961705F666C6173685F696E33
:10D3700074662E63000000000120800270470000E8
:10D3800010B5272804D2064980000858002805D186
:10D39000EC2204A10020FFF7EFFA0AA010BD000064
:10D3A000903001002E2E5C2E2E5C2E2E5C736F753D
:10D3B0007263655C6461706C696E6B5C6572726FE0
:10D3C000722E63000000000001460120272901D2CF
:10D3D0000148405C7047000001F0FF1FF3B581B0C9
:10D3E0000446009000E0641C2078402802D0002809
:10D3F000F9D164E06078622848D012DC522854D019
:10D4000008DC422842D0442849D0482841D04D2841
:10D4100017D134E054283FD0552833D0562810D1A6
:10D4200040E0722841D006DC642838D0682830D02B
:10D430006D2806D123E074282ED0752822D07628B6
:10D4400030D020A52046FAF7ADFF07462846FAF768
:10D45000A9FF0646A019029B009AC119D218891E7D
:10D4600091422BD2BA1EA11CFBF786F83246294600
:10D470002046FBF71DF820780028B5D11FE000F00A
:10D4800053FF01E000F058FF0546DBE700F0FAFE2D
:10D49000FAE700F027FFF7E700F04AFFF4E700F0B3
:10D4A0001DFFF1E700F050FFEEE70848807A002802
:10D4B00002D0064D0A35C5E705A5C3E7E419009873
:10D4C000201AFEBD4552524F520000002830010084
:10D4D00068747470733A2F2F6D6265642E6F726773
:10D4E0002F6465766963652F3F636F64653D4055C2
:10D4F0003F76657273696F6E3D40563F7461726727
:10D5000065745F69643D405400000000704700008E
:10D51000F8B51E4615460C46074605F02BFB2C4871
:10D520000178032912D001462039022C0FD0002C9B
:10D530001FD0012C0AD10A68AA4207D1807800289E
:10D5400033D00020421E08608A608861F8BD0868F8
:10D55000A842FBD1304605F057F80446304605F0A6
:10D5600059F80646384602F0B7FE034622463146D1
:10D5700017E0384602F0B0FE0328E7D0304605F049
:10D5800041F88007E2D4384602F0A6FE074630464E
:10D5900005F03AF80446304605F03CF801463B46B3
:10D5A0002246284604F02CF8F8BD094828220949EB
:10D5B0002038FAF78DFE03F0F1FC07488178012945
:10D5C00003D14178022900D1817003F0F1FCF8BD4C
:10D5D000BC02002090310100FCF0FF1FF7B51C4E8B
:10D5E0000446B0785502174600280BD12946019809
:10D5F00002F030FE032802D0214603F0ADFFB078E0
:10D60000002812D0124920394868A0420DD8C868B5
:10D61000A0420BD0A04208D90869401C00D10C617F
:10D620000869A04200D204460C61FEBDC8692A46C2
:10D630008018C861E019C860F078002803D0002085
:10D6400004F02EF8FEBD2046019903F02FFFFEBD29
:10D65000BC020020F0B585B018A1096804910378D8
:10D66000002104AA545C9C4226D0491C0329F9D30A
:10D6700013A10A688E6896464A68CD6800239446CE
:10D68000C25C714664466F46039552C711466139C4
:10D69000192911D9202A01D2052A0DD100216C4661
:10D6A000675C974208D0491C1029F9D35B1C0B2BEF
:10D6B000E6D3012005B0F0BD0020FBE7E500200027
:10D6C000222A2B2C2E2F3A3B3C3D3E3F5B5C5D7C5F
:10D6D00010B50448FAF7A1FF002801D0012010BDC1
:10D6E0000020FCE71830010070B50446204600F029
:10D6F0001AF80546002D00D070BD0449024809689B
:10D70000884700BFF8E700000C3000F0D4F2FF1F9C
:10D7100001680122920211430160BFF36F8FBFF3D2
:10D720004F8F70477047002807D0C069002802D08B
:10D730000068022803D06D20704704207047002045
:10D74000704710B5002806D05B1E194201D11A425D
:10D7500003D0652010BD042010BD03688B4204D89F
:10D76000406889181818884201D2662010BD002030
:10D7700010BD00000349884201D06B207047002093
:10D78000704700006B66656B10B50C4C7021217002
:10D79000FFF7C9FF002807D10949204609688847D3
:10D7A0002078810601D5672010BDC10601D568200B
:10D7B00010BDC007FCD0692010BD00000000024071
:10D7C000D0F2FF1F70B50E4D00202C78002C0FD02A
:10D7D00000212970A978002901D000F0ABFB022CB0
:10D7E00005D06978032902D0002800D1242070BD1B
:10D7F000FF22443203A10020FFF7BEF8022070BDD3
:10D80000A8F0FF1F2E2E5C2E2E5C2E2E5C736F75E3
:10D810007263655C6461706C696E6B5C6472616795
:10D820002D6E2D64726F705C666C6173685F6465E9
:10D83000636F6465722E6300FEB51C460546302991
:10D8400001D3012000E00020412217A1FFF794F846
:10D8500029460C2220316846FAF72AFE1F4E002C7A
:10D8600001D1002030711E49019888420BD11D4919
:10D870000098884201D10220FEBD1A49FC39884235
:10D880000FD10120FEBD284604F086FD002804D0FB
:10D89000002C04D10120307101E0002C01D00320C4
:10D8A000FEBD0020FEBD00002E2E5C2E2E5C2E2E16
:10D8B0005C736F757263655C6461706C696E6B5CE0
:10D8C000647261672D6E2D64726F705C666C61733B
:10D8D000685F6465636F6465722E6300A8F0FF1F64
:10D8E000019996978F9E939BFFB581B006460024C1
:10D8F00004982546002813D00A98002810D00499CF
:10D90000002008600A9907460860FFF76AFC0028B3
:10D9100012D00120C003022E04D0032E0AD03FE013
:10D920006B2253E00399002904D00299814201D06F
:10D930001B2436E0074610E0FFF755FC00282FD0E7
:10D94000012E02D0032E0AD02AE00398002804D02A
:10D950000298002801D01A2423E01F4819E01F482C
:10D96000FAF75BFE00281BD005460C3506E028467A
:10D970000830FAF752FE01280DD014352846FAF780
:10D980004CFE0028F3D1281DFAF747FE0028EED1FF
:10D990001348056805E02846FAF73FFE0746F7E713
:10D9A0001C24FFF799F9002801D1012E04D0002C86
:10D9B00004D0204605B0F0BD1C24FAE7002D04D0A9
:10D9C000049807600A980560F3E7AD2205A10020DE
:10D9D000FEF7D2FF0220EDE78C3101001830010084
:10D9E000503101002E2E5C2E2E5C2E2E5C736F7536
:10D9F0007263655C6461706C696E6B5C64726167B4
:10DA00002D6E2D64726F705C666C6173685F646507
:10DA1000636F6465722E6300F7B51E490646487849
:10DA20000025012804D0022805D0032830D105E0C4
:10DA30000125ED0326E07F25AD0223E008790028CB
:10DA400026D01548FAF7E9FD002821D004460C3409
:10DA50000CE0B74209D8201DFAF7DFFDB04204D32D
:10DA6000201DFAF7DAFD05460AE014342046FAF7DD
:10DA7000D4FD0700EDD1201DFAF7CFFD0028E8D135
:10DA8000002D05D002983018A84201D30120FEBD18
:10DA90000020FEBDA8F0FF1F1830010010B50D4C8E
:10DAA0002078002806D0BC220BA10020FEF764FFDE
:10DAB000022010BDFF2230211448FAF785FD012015
:10DAC000207000206070A060E0602061A070E070B5
:10DAD00010BD0000A8F0FF1F2E2E5C2E2E5C2E2EF7
:10DAE0005C736F757263655C6461706C696E6B5CAE
:10DAF000647261672D6E2D64726F705C666C617309
:10DB0000685F6465636F6465722E630020F8FF1FB1
:10DB1000F7B5434F0646387884B01546012807D03C
:10DB2000D12240A10020FEF727FF022007B0F0BD60
:10DB3000F878002803D1FE6001203E61F870B878C3
:10DB4000002857D139698E4201D1012000E0002020
:10DB50004919396100282FD0B86830210C1AAC421D
:10DB600000D914463C49224608180599FAF7A0FC4A
:10DB7000B8682D1B0019B860059936190919059167
:10DB800030282AD316D00020F32226A1FEF7F4FE77
:10DB900001233148FA68B968FFF74EFE787001A892
:10DBA000009002AB01227878F968FFF79DFE00280B
:10DBB00027D103E00120E7E70320EFE7B87801244D
:10DBC000FF2260400D3217A1FEF7D6FE019800F04B
:10DBD00043F9002815D1BC7002E0B878002813D0B2
:10DBE0001D49BA68F86800F093F8002809D1B878A0
:10DBF000002809D02A463046059900F089F8002807
:10DC000002D00321397091E72A4630460599FFF783
:10DC100003FF00288AD002203870132086E7000016
:10DC2000A8F0FF1F2E2E5C2E2E5C2E2E5C736F75BF
:10DC30007263655C6461706C696E6B5C6472616771
:10DC40002D6E2D64726F705C666C6173685F6465C5
:10DC5000636F6465722E630020F8FF1F10B5EFF349
:10DC60001081CC07E40F72B6FBF7A2FB002C00D1A9
:10DC700062B610BDFEB5174F05467E787C68AE4291
:10DC800022D0002E0ED0201DFAF7C7FC00210091F3
:10DC90000B460191014620463246183002F08AFBBD
:10DCA000002813D0002D0ED02046FAF7B6FC002134
:10DCB00001910B460146009520461830FA6802F0A3
:10DCC00079FB002804D07D700020FEBD0C20FEBD35
:10DCD0000B20FEBD6CF0FF1F70B50E46050014460C
:10DCE00013D020211046FAF796FC2660E8686060A1
:10DCF000A9686868FAF7AAFCA0600420E0602061C7
:10DD00006061A061E061002070BD042070BD000072
:10DD1000F7B5424E04467078002582B017460128B8
:10DD200007D078223EA10020FEF726FE022005B093
:10DD3000F0BDF07800280AD1204602F033F9050042
:10DD400002D00220707066E00120F07074613348E8
:10DD5000816820460091FAF779FC3048661A0099EC
:10DD600040690090FAF772FC0098401A864208D089
:10DD7000204600F03FF9050003D0284902204870F2
:10DD800049E02648016920460091FAF75FFC2348E4
:10DD9000661A009940690090FAF758FC0098401AFA
:10DDA000864204D0204602F0FDF80500E5D11B4E66
:10DDB000B16870684018A04204D8204600F01AF9F3
:10DDC0000500DAD1002F24D03169F0684018A04254
:10DDD00004D8204602F0E6F80500CED10F49486885
:10DDE0008968201A0E1AB74200D23E4619493246B7
:10DDF00008180399FAF75CFB002E08D000200749A9
:10DE0000A419887003988019BF1B0390CFE70120E5
:10DE1000F5E702484461284689E70000BCF0FF1F8F
:10DE20002E2E5C2E2E5C2E2E5C736F757263655CDD
:10DE30006461706C696E6B5C647261672D6E2D64D9
:10DE4000726F705C666C6173685F6D616E6167654F
:10DE5000722E630050F8FF1F70B5244D0446687899
:10DE6000002801D044222FE0002C2CD0606800282C
:10DE700029D0A068002826D0E068002823D0206997
:10DE8000002820D0606900281DD0A06900281AD081
:10DE9000E069002817D00121FF2289021448FAF70F
:10DEA00093FB0126AE700020E8706860A860E8600F
:10DEB0002861AC61686120688047040009D1287836
:10DEC000002807D010E04A220AA10020FEF754FDE6
:10DED000022070BDA86900698047040004D0A869C9
:10DEE00040688047204670BD6E70FBE7BCF0FF1FA6
:10DEF00050F8FF1F2E2E5C2E2E5C2E2E5C736F753D
:10DF00007263655C6461706C696E6B5C647261679E
:10DF10002D6E2D64726F705C666C6173685F6D61ED
:10DF20006E616765722E63000149087070470000DA
:10DF3000BCF0FF1F70B5164C00256078002802D099
:10DF4000012807D00AE0C92212A10020FEF714FD23
:10DF5000022070BD002000F04DF80546A069406821
:10DF6000804706460121FF2289021748FAF72CFB59
:10DF700001200021A070E1706160A160E160216179
:10DF800061616170002E01D0304670BD284670BDC1
:10DF9000BCF0FF1F2E2E5C2E2E5C2E2E5C736F7538
:10DFA0007263655C6461706C696E6B5C64726167FE
:10DFB0002D6E2D64726F705C666C6173685F6D614D
:10DFC0006E616765722E630050F8FF1F10B5EFF3A6
:10DFD0001083DC07E40F72B6FBF7E2FB002C00D1E4
:10DFE00062B610BD8021017001780906FCD570472A
:10DFF0007047000070B50E4D0646A8780024002832
:10E0000008D1A8690B498368AA68686898470446DC
:10E010000120A870FF220748A968FAF7D5FA304610
:10E02000A968FAF713FB701A6860204670BD0000FB
:10E03000BCF0FF1F50F8FF1F10B50748FAF7EDFAC4
:10E04000002805D0FF309D30FAF7E7FA002801D10B
:10E0500001480C3810BD00001830010010B5094807
:10E06000FAF7DBFA002806D0FF30A13041780278B9
:10E070000802104305D103481038C178827808029D
:10E08000104310BD18300100034601220149002051
:10E0900018470000C4020020F8B505461248FAF7F8
:10E0A000BCFA04460C34114F10E0AE420DD8201DCE
:10E0B000FAF7B3FAA84208D32046FAF7AEFAF860A6
:10E0C00020461030FAF7A9FAF8BD14342046FAF7C2
:10E0D000A4FA0600E9D1201DFAF79FFA0028E4D13E
:10E0E000BC68002CE8D1F8BD183001006CF0FF1FAF
:10E0F000024800698007C017401C704740F00F407D
:10E100000020704708B51A48816B1F225202114344
:10E11000816318498015086108610861164A5060DA
:10E120008860002000F03AF8002000F02DF8002070
:10E1300000F03EF811480168042319430160426968
:10E1400010210A43426142690A43426142690A431B
:10E15000426141691943416108488038416902229E
:10E160009143416106480090401E0090FCD108BDDB
:10E170000080044000C0044000A00440C0F00F40F4
:10E1800040420F007047000010220349012801D0CF
:10E190004A6070478A607047C0F00F401022034900
:10E1A000012801D04A6070478A607047C0F00F4074
:10E1B00010220349012801D04A6070478A607047E5
:10E1C000C0F00F40092800D927303030C0B2704766
:10E1D0001CB501AA69460A48FBF7C0F8002807D019
:10E1E0000198402805DD322206A10020FEF7C4FB7D
:10E1F0001CBD40220020009903F03CFF1CBD000024
:10E20000C02400202E2E5C2E2E5C2E2E5C736F758B
:10E210007263655C7573625C6869645C7573626483
:10E220005F757365725F6869642E630010B50F498E
:10E23000002008600E4908600E4908600E49086019
:10E240000E49FEF741FF0949086001200C49C0034F
:10E25000FEF73AFF0649086001217F20890280020B
:10E26000FEF732FF0449086010BD00002CF0FF1FCC
:10E2700030F0FF1F34F0FF1F38F0FF1FFC7F00005D
:10E28000FC7B0100004870473CF0FF1F012000218B
:10E29000096A054A914200D000200021496A034AD8
:10E2A000914200D000207047939D939B01999697CF
:10E2B00000B5FFF7EBFF002800D100BD0020806A09
:10E2C000FBE7000001480068704700002CF0FF1FCA
:10E2D000014800687047000030F0FF1F0048704799
:10E2E000ACF6FF1F004870476AF6FF1F0120C1030C
:10E2F000096A064A914200D000200121C903496AF7
:10E30000034A914200D00020704700008F9E939BEB
:10E310000199969700B5FFF7E9FF002800D100BDED
:10E320000120C003806AFAE7004870475DF6FF1FCE
:10E33000004870478BF6FF1F004870472CF6FF1F00
:10E3400000487047B5F6FF1F0048704746F0FF1FB2
:10E3500010B5FFF76BFF054800F0B6FF01F058FD60
:10E3600001F0DEFE01F0B0FE10BD00000CF6FF1F54
:10E3700010B5134C2078002806D0622211A100208D
:10E38000FEF7FAFA022010BD002211461046FBF7F4
:10E39000CBF9002801D01D2010BD00206070A070B6
:10E3A000E070A060E0602071206160610121A061E7
:10E3B00089021248FAF72DF901202070002010BDC3
:10E3C000D8F0FF1F2E2E5C2E2E5C2E2E5C736F75E8
:10E3D0007263655C6461706C696E6B5C64726167CA
:10E3E0002D6E2D64726F705C6961705F666C617315
:10E3F000685F696E74662E630000000050FCFF1FAA
:10E4000010B50024FFF72AFE0D4A0E4B11680029B3
:10E4100014D10AE00988002905D0814203D1A00067
:10E420001858106006E0641CE4B2A1005958002995
:10E43000F0D11068002801D10348106010BD000021
:10E44000D0F4FF1FD4F4FF1FFC41010030B50023BE
:10E4500005E0DD000C46EC40C4545B1CDBB293428B
:10E46000F7D330BDF7B504462F4801250078ED03FA
:10E4700082B01746012808D0FF227A322BA1002053
:10E48000FEF77AFA022005B0F0BDAC4201D322209B
:10E49000F9E7FEF7A8FE002844D02E1B301FB84233
:10E4A00001D93A4600E0321F1F4803998069FEF700
:10E4B0002FFE1D498861009001208002844207D20E
:10E4C00028483A4600190399F9F7F2FF0020DAE7E5
:10E4D000E019A84226D103988519281FFAF79DF85C
:10E4E0000102203DE87F090A0006014300980E4D15
:10E4F000884201D02620C6E739462046039AFFF716
:10E5000065FD002801D01F20BDE7012292021549B8
:10E510000020FEF725FE0446FFF788FE0120687004
:10E520002046B0E72520AEE7D8F0FF1F2E2E5C2E48
:10E530002E5C2E2E5C736F757263655C6461706C0B
:10E54000696E6B5C647261672D6E2D64726F705CB6
:10E550006961705F666C6173685F696E74662E6373
:10E560000000000050FCFF1F70B505461048012454
:10E570000078E403012807D0FF22BC320DA100205F
:10E58000FEF7FAF9022070BDA54201D3222070BD2A
:10E59000FEF729FE002801D0002D01D0252070BDF6
:10E5A000FF22002001322146FEF7DAFD70BD000097
:10E5B000D8F0FF1F2E2E5C2E2E5C2E2E5C736F75F6
:10E5C0007263655C6461706C696E6B5C64726167D8
:10E5D0002D6E2D64726F705C6961705F666C617323
:10E5E000685F696E74662E63000000000246880052
:10E5F000064910B540188038C06F002804D0114675
:10E6000001F0DAF901F0C8F910BD00007C22002009
:10E6100001200749C003886001F0F8FB00F0CEF943
:10E6200000221146034800F01BFA00F0CDF9FEE786
:10E6300000ED00E091E60000024901224A700871F5
:10E64000704700004CF0FF1F024901220A70C87099
:10E65000704700004CF0FF1F024901228A70487188
:10E66000704700004CF0FF1F10B503480121C9029C
:10E67000C06800F0C9F910BD4CF0FF1F10B5034889
:10E680000421C06800F0C0F910BD00004CF0FF1F6D
:10E690000EB516200127009000203E463D46019011
:10E6A000FEF72AFBFEF78AF900F0D2F99D4CE060F4
:10E6B000FFF728FD3846FFF771FD3046FFF764FD90
:10E6C0002846FFF775FDFAF7DBFD97484178027899
:10E6D00008021043012800D00020D72293A1FEF7A2
:10E6E0004BF991486A30F9F798FF002800D080472D
:10E6F000FFF786FE98480068002803D0C06800280D
:10E7000000D0804788480C300290F9F786FF8007D8
:10E7100002D5012002F066F80298F9F77EFFC007E3
:10E7200002D00120FFF700FCFFF712FE03F048FDC6
:10E73000FEF798FB00283ED0002004F097F8002058
:10E7400003F054FC77480121C1710B200023029093
:10E750001A46824800F0ACF9032100F0B1F900221A
:10E76000D24300217E4800F063F984B2A00508D5A9
:10E770006C488079002802D0012000F00DF9FCF7E8
:10E7800083FC600702D5022002F03EFEE00614D5AD
:10E79000032002F039FE0020FFF7F4FC002003F014
:10E7A00025FC0020FFF7FAFC0020FFF7EDFC00201D
:10E7B000FFF7FEFCFEE70120BFE7A00602D503201D
:10E7C00002F022FE200501D5FEF72AF9E00738D035
:10E7D0005A2004F079F85348C079002831D0012834
:10E7E0000CD0032819D005282BD14E490020C87120
:10E7F000FFF7C8FC002003F0F9FB22E00298002894
:10E8000002D0401E02901CD1012003F0EFFB4548CE
:10E810000321C1711620009013E003F0DFFB0028F4
:10E8200006D00120FFF7AEFC3E480221C17108E08E
:10E830000098002802D0401E009002D10120FFF76E
:10E84000A1FCA0078BD50198002804D0FFF750FC4D
:10E8500000280ED012E0FFF74BFC00280ED04148F4
:10E860000068C0698047002808D102F0CDFD012072
:10E8700003E0022002F0C8FD00200190294C20781E
:10E8800000280AD0E078012825D0022823D00127CB
:10E89000002020703846FFF781FCA07800280AD0BD
:10E8A0006079012824D0022822D001250020A07000
:10E8B0002846FFF77DFC6078002800D14FE72079DB
:10E8C000012822D0022820D0012600206070304686
:10E8D000FFF75AFC43E7012F01D0012700E0002792
:10E8E000002FD7D00128D5D100202070E070D1E7CB
:10E8F000012D01D0012500E00025002DD8D00128F0
:10E90000D6D10020A0706071D2E7012E01D001267F
:10E9100000E00026002EDAD00128D8D10020607057
:10E920002071D4E74CF0FF1F083001002E2E5C2E22
:10E930002E5C2E2E5C736F757263655C6461706C07
:10E94000696E6B5C696E746572666163655C6D614E
:10E95000696E2E6300000000D0F4FF1F81140100D7
:10E96000370A0000503101000149887170470000EA
:10E970004CF0FF1F10B5FFF791F810BD10B5FF2147
:10E9800004460231F9F745FE00F032FD0020207008
:10E99000FFF784F810BD000080B5034F80B2BC467D
:10E9A00000DF002080BD000031F5000080B5024F7F
:10E9B000BC4600DF80BD000009FD000001490020C9
:10E9C00008607047A4F4FF1F0020704780B5034F14
:10E9D00089B2BC4600DF002080BD0000BDF8000009
:10E9E00080B5044F0248BC4600DF014880BD0000EE
:10E9F0008820002005F8000080B5024FBC4600DFEB
:10EA0000002080BD15F80000B0B50C460146EFF3BC
:10EA10000380C00603D0A0B2FFF7E8FD03E0034F78
:10EA2000A0B2BC4600DF2046B0BD000095F5000056
:10EA300080B5054F91B280B20022BC4600DF034F83
:10EA4000BC4600DF80BD0000F1F500003DF5000090
:10EA500080B5024FBC4600DF80BD0000FDFD000018
:10EA6000F8B50E4C06462068002500280CD000237F
:10EA70000B4F1A460B213046BC4600DF0546206886
:10EA8000401C20602846F8BDF9F764FB074F054A93
:10EA900005493046BC4600DFF1E70000A4F4FF1F43
:10EAA00081FD0000E01C00200A20030095FB00000F
:10EAB0000146024A0020516070470000A4F4FF1F85
:10EAC00080B50548084F81600023044A0449054881
:10EAD000BC4600DF002080BDA4F4FF1F0020002002
:10EAE0000B88000015FD000081FD0000012805D005
:10EAF000022805D003280BD0C72202E0BB2200E089
:10EB0000BF2204A10020FDF737FFFBF7B1F9FEE7B4
:10EB1000C322F6E72E2E5C2E2E5C2E2E5C736F75B4
:10EB20007263655C72746F735C5254585F436F6EAE
:10EB30006669672E63000000FEE700000748016871
:10EB40000748416100218161072101610548016A8F
:10EB5000FF2212061143016240177047D4410100A1
:10EB600000E000E000ED00E070477047FFB583B0C3
:10EB7000054604980E9C281800900020854F2060C0
:10EB8000F878854E00281BD00020F870701E02789F
:10EB9000011D0698F9F78CFC701E00780699411843
:10EBA0000691216808182060786871783278000C26
:10EBB0000902000411430843711E09784018786067
:10EBC000CCE028780A2829D00D28FCD03A281CD07F
:10EBD0003978002976D0FEF7FDFA02076E49787879
:10EBE000491E0B5C120F1A430A54401CC0B27870C5
:10EBF00009780291491D884263D3674A0021521E59
:10EC0000137808465B1D9C460EE063482521401E94
:10EC1000F9F7FFFC002038707870B8709DE0135C45
:10EC20005918401CC9B2C0B28445F8D8002901D097
:10EC3000042698E0B878002843D10120B870707895
:10EC400031780002084340BA3070010A71700190B7
:10EC50005148401EC078002806D0012833D0022831
:10EC600033D0042874D14BE04B492522491E881823
:10EC7000F9F71EFC7868019A010C090411438142DE
:10EC800003D00120F87002266DE04349029AC91CA6
:10EC90000698F9F70DFC40480699401E0078411887
:10ECA0000691216808182060786871783278000C25
:10ECB00009020004114308433749491E09784018E6
:10ECC000786045E03AE001264DE021680C98FF228B
:10ECD000411A0698F9F778FC20687968091A0D98A6
:10ECE00001600098411B0498411A059801602A4868
:10ECF000401E0179407909030001014379601AE05F
:10ED000021680C98FF22411A0698F9F75DFC2068EB
:10ED10007968091A0D9801600098411B0498411AFE
:10ED2000059801601C48401E417902790802104391
:10ED300040BA00047860022007B0F0BD7978252938
:10ED400025D2FEF747FA144900017A78491E885403
:10ED5000387800281BD0002038706D1C0098854240
:10ED600000D02EE7002621680C98FF22411A069851
:10ED7000F9F72AFC20687968091A0D980160009853
:10ED8000411B0498411A059801603046D4E70120E0
:10ED9000E2E70000F4F0FF1F5100002010B5044826
:10EDA00002490068F9F74AFC10BD0000C8F2FF1FD5
:10EDB0000430010070B5134D0646EFF31080C40710
:10EDC000E40F72B62846FAF7F3FA002C00D162B6C7
:10EDD000002816D1FF2210210B48F9F7F5FB092274
:10EDE00031460948F9F764FBEFF31080C407E40FDC
:10EDF00072B6054A10212846FAF7D2FC002C00D141
:10EE000062B670BD00FC010028230020F7B504465F
:10EE1000012084B0C003434F029038781646012881
:10EE200005D0A22240A10020FDF7A6FD41E0FF2170
:10EE300001318800009001912046F9F707FC022576
:10EE4000002901D0AB222FE00198864205D301466C
:10EE50003046F9F7FBFB002901D0B22224E020461E
:10EE60000099F9F7F3FB00988919814201D9B92279
:10EE70001AE0B87800280DD1F878002808D0B968D1
:10EE80008C4203D3F8680818A04203D8C7220BE0CD
:10EE9000C12209E03979384600290DD07A693969EB
:10EEA0008918A14208D0CF221FA10020FDF764FDE0
:10EEB0003D70022007B0F0BD7F218902A7198C4266
:10EEC00005D20121C9038F4201D9002100E00121AF
:10EED000002910D0134801210171466104613246B6
:10EEE00020460599FFF7BEFA252807D00028E1D073
:10EEF0000C490D70DEE705701F20DBE73146204628
:10EF0000059AFFF763F8002801D00648F3E7029856
:10EF1000874204D3FFF78AF9024901204870002094
:10EF2000C8E70000D8F0FF1F2E2E5C2E2E5C2E2E80
:10EF30005C736F757263655C6461706C696E6B5C49
:10EF4000647261672D6E2D64726F705C6961705FB1
:10EF5000666C6173685F696E74662E630000000002
:10EF6000FF2001307047EFF31082D207D20F72B644
:10EF700003680B400360002A00D162B67047EFF3CC
:10EF80001082D207D20F72B603680B430360002AC7
:10EF900000D162B67047EFF31082D207D20F72B67B
:10EFA00003684B400360002A00D162B6704700003E
:10EFB00070B514460E46054600190121400289022B
:10EFC000884207D9992292000AA10020FDF7D4FCBB
:10EFD000002070BD012149023046F9F71AFB002DCF
:10EFE00006D111481149006942013046F9F760FA2B
:10EFF000600270BD2E2E5C2E2E5C2E2E5C736F7503
:10F000007263655C6461706C696E6B5C647261678D
:10F010002D6E2D64726F705C7669727475616C5FB1
:10F0200066732E630000000014F1FF1FC809002062
:10F0300010B5012464020B46002801D0002010BD49
:10F04000224603491846F9F733FA204610BD00005E
:10F0500008070020F8B50C4600210E460091002854
:10F0600001D00020F8BD31480078012842D00228A4
:10F0700042D0002720462EA103F04AF90546601928
:10F080002EA103F045F9451960192E4903F040F906
:10F09000451960192CA103F03BF9451960192BA102
:10F0A00003F036F9214945196019498803F039F907
:10F0B0004519601924A103F02BF94519002F0ED032
:10F0C000601924A103F024F945196019394603F0A9
:10F0D0001FF9451960191CA103F01AF94519684672
:10F0E000FDF7C6FE07001FD0009800281CD060194D
:10F0F0001BA10EE01DA7BDE71FA7BBE7B00000994D
:10F10000761C0958F6B2601903F0DCF8451960194D
:10F110000DA103F0FDF84519BE4205D22846012194
:10F120000A3049028842E9D32846F8BD0CF1FF1F96
:10F130004173736572740D0A0000000046696C65C6
:10F140003A200000C40400200D0A00004C696E65DE
:10F150003A200000536F757263653A20000000008A
:10F1600048657864756D70730D0A0000426F6F74A6
:10F170006C6F6164657200004170706C69636174EA
:10F18000696F6E0010B50A46002801D0002010BD3E
:10F1900001214902104602F037FC10BDF8B50D46BA
:10F1A000044603F089FB0646FEF7EAF807463046B8
:10F1B000FEF70AF90646002C01D00020F8BD2846CB
:10F1C0001B4903F0A5F804462819394603F0A0F8B6
:10F1D0000419281917A103F09BF8154904192819D7
:10F1E000C91F03F095F8041900270120009014E0CE
:10F1F0000098002804D128190FA103F089F80419F8
:10F20000F00708D00D49B8000958281903F080F814
:10F2100004190020009076087F1C002E01D0052FD5
:10F22000E6D3281903A103F073F80019F8BD000014
:10F23000BF3101000D0A00002C200000283301001E
:10F2400070B50C46002801D0002070BD01256D026C
:10F2500029462046F9F7DDF90648F9F7A3F80246F2
:10F2600004492046F9F724F929462046FEF7B6F866
:10F2700070BD0000C7310100F8B5094D06460F46C4
:10F280002846F9F78FF80446002E01D00020F8BD7B
:10F29000024629463846F9F70BF92046F8BD00002A
:10F2A000D44C010010B5012464020B46002801D0A3
:10F2B000002010BD224603491846F9F7F9F8204608
:10F2C00010BD00000805002004490A6A0260CA69EE
:10F2D0004260896981600021C160704740800440BC
:10F2E00010B5084654022146F9F793F9204610BD9F
:10F2F00070B5234D00246878A978E443884201D092
:10F30000012000E00020FF22F9321EA1FDF734FBAE
:10F310006878022804D0002816D0012818D020E0F0
:10F320002548FF240078F53400281AD0012809D098
:10F33000022816D0032814D0204A12A10020FDF77D
:10F340001BFB0EE01E4C0CE0A878022808D008E059
:10F35000A878022802D0002802D002E0194C00E070
:10F360000024601C05D1154A06A11032FDF704FBEC
:10F370000024A868A04201D9012070BD002070BD02
:10F38000FCF0FF1F2E2E5C2E2E5C2E2E5C736F75F4
:10F390007263655C6461706C696E6B5C64726167FA
:10F3A0002D6E2D64726F705C7666735F6D616E6139
:10F3B0006765722E63000000BC0200200A02000094
:10F3C000204E0000C409000070B50346002002462C
:10F3D000012509E0DC0704D08E1A2C46761EB440C5
:10F3E00020435B08521CD2B28A42F3D370BD0000A6
:10F3F00010B525210748F9F70CF9064825212530D5
:10F40000F9F707F9044800214160017041708170EB
:10F41000C17010BD50000020F4F0FF1F0146EFF353
:10F420001080C207D20F72B60868002801D00368A6
:10F430000B60002A00D162B67047000070B50D461F
:10F4400000280FD00849094C884204D2226801469E
:10F45000104600F0D1FA20684570054800F0FBF82E
:10F4600000F090FB70BD0000FFFF0000B8F4FF1F2C
:10F47000942000207047000070B51B4EF0680028F3
:10F4800031D0B08A401EB082002526E0A068002856
:10F4900008D0616841606068002802D0A16881607E
:10F4A0006560A56010482146183800F0CDFAA08AA2
:10F4B000B0826078042804D10C49E08A0988401899
:10F4C000A0820120607020210855E068F060E068AB
:10F4D000002801D00661E5602561B08A002802D1CC
:10F4E000F468002CD2D170BDAC200020C0F4FF1F06
:10F4F00070B504000ED00C4DA178286801268278E2
:10F5000091420BD900F0BEFA28684670204600F000
:10F5100039FB70BD054800F09EF8F8E7667021469B
:10F52000024800F091FA70BDB8F4FF1F942000204B
:10F5300010B50321FFF782FF10BD000001480068ED
:10F54000408B7047B8F4FF1F10B50446008B08438A
:10F5500020836278618B062A15D0052A12D10842D1
:10F5600010D00A460240628388432083204600F080
:10F57000ABFA012060700221202001552146044889
:10F5800000F062FA10BD0A468243EDD010BD0000C3
:10F59000942000200246880070B514494018803835
:10F5A000C46F002C1DD0208B104320836178658BA5
:10F5B000062917D0052914D1284212D02946014026
:10F5C0006183A8432083204600F07EFA208B02212D
:10F5D000A843208301206070202001552046FFF7BA
:10F5E00087FF70BD29468143EBD070BD7C2200208F
:10F5F00070B503460D480D460468002A208B08D0DC
:10F600001946814301D0062109E098432083022056
:10F6100070BD0146194001D06183F6E7052163837F
:10F620002846FFF70BFF012070BD0000B8F4FF1F54
:10F63000814202D342688A4201D801207047EFF329
:10F640001082D207D20F72B603680B60016000D13E
:10F6500062B60020704701464068002342684A6055
:10F660000A78022A05D0012A03D0032A01D0436078
:10F6700070474268002A01D0916043608360704700
:10F6800070B5044615460020207001226270A170FA
:10F690006060A060E0602061A082E0822083234659
:10F6A0006083203318705870608C002803D10448A0
:10F6B000FFF7B4FEA0622946204600F005F870BDB1
:10F6C000C02100207047000030B5428C920803D161
:10F6D0000E4A12881204920C836A92009B185A07F1
:10F6E00000D51B1F01221206403BDA6300229963FA
:10F6F00014469500521C5C510E2AFAD3C2691A6254
:10F700004362C162806A0249016030BDD04101009C
:10F71000A52E5AE20349044A0968C8821288801853
:10F7200088827047B8F4FF1FC0F4FF1F10B5084867
:10F73000016808488A8A0088CB8A101AD21880B2D9
:10F740008A82010402D40421FFF778FE10BD000074
:10F75000B8F4FF1FC0F4FF1FF8B504464068002648
:10F760000F46002805D06078022818D0A08900280C
:10F770002FD0A089E18988423ED2208980000019DB
:10F78000076172B6A089401CA08162B62089401C26
:10F7900080B22081E189884200D12681F8BD66705F
:10F7A0002046FFF758FF0546203006702189E8699A
:10F7B00089000919086172B6A089401CA08162B64F
:10F7C0002089401C80B22081E18988420AD12681AB
:10F7D00008E02046FFF73FFF0546C06904210760A7
:10F7E0002020415501206870284600F06DF9294617
:10F7F000034800F029F9F8BD0320FFF777F9F8BDB9
:10F80000942000200321017000214170418041605B
:10F8100081607047F8B504464088002804D0254E22
:10F82000A1683268914201D0FF20F8BD401E00045B
:10F83000000C60803CD13168607888706168012775
:10F84000002928D02046FFF706FF05460521203075
:10F850000170284600F038F96780A560A8786070CC
:10F860001548316840688A788078824201D32846FA
:10F870000AE0114800F0E8F829460F4800F0E4F8E3
:10F88000306847706F7011E0FFF732FE316800207A
:10F89000203108700CE0084949688A783168824252
:10F8A00006D9054800F0D0F8306847700020EBE733
:10F8B0000020F8BDB8F4FF1F9420002070B50E465C
:10F8C000184D044641882868002907D0A168814264
:10F8D00008D16088401C6080002070BDA0608078E6
:10F8E0006070F6E7002E0FD062788078824203D2F3
:10F8F0008870A06800F0D0F86068002806D0204624
:10F90000296800F0A1F808E0012070BD2868606057
:10F910002968002048602868846009213046FFF784
:10F920008DFDF1E7B8F4FF1F70B51848012102689A
:10F930005170006800F0A6F8154D6C7813E0E000F7
:10F94000411948680278002A17D0012A1AD000F01D
:10F95000EBF8E878641C844200D1002472B6A878E1
:10F96000401EA87062B6A8780028E8D16C700948DB
:10F97000FFF771FE00F006F970BD098989B2FFF743
:10F98000E3FDE6E78968FFF7E7FEE2E7B8F4FF1F6B
:10F99000582200209420002005480178002902D038
:10F9A00001214170704701200249000748607047FB
:10F9B000B0F4FF1F00ED00E0F8B50E4EF778B41C70
:10F9C000354672B6B278BA4207D2521C22702A78F3
:10F9D000531CBB4200D100232B7062B6F3789342D4
:10F9E00004D9D200921991605060F8BD0220FFF74F
:10F9F0007DF8F8BD5822002010B5124AD368002BBC
:10FA000017D013469B8A04E0002C12D02246A48A09
:10FA1000E318D4688B42F7D3C460D0600261C46835
:10FA2000002C00D02061591A8182908A401A90825D
:10FA300010BD0024C460D060C91A02619182848222
:10FA400010BD0000AC20002030B502780023022A4F
:10FA500003D0012A01D0032A00D101238C7800E0D1
:10FA600010464268002A02D09578A542F8D24A6032
:10FA70004160002B04D0002A00D09160886030BD26
:10FA80000020FBE703494A68426000228260486028
:10FA9000704700009420002010B583680446002BB6
:10FAA00005D1607801280CD1064B03E09B681878DB
:10FAB0000028FBD0204600F01DF821461846FFF72D
:10FAC000C3FF10BD9420002010B5016900290FD09C
:10FAD000C268CA60C3680022002B07D08B8A848A60
:10FAE0001B198B82C3681961C26000E08A820261BF
:10FAF00010BD00008168002907D042684A60416853
:10FB0000002901D0806888607047064906E04A688D
:10FB1000824202D140684860704711460029F6D100
:10FB2000704700009420002010B5416800290ED0D5
:10FB3000FFF791FD0446FFF7C7FF01206070032126
:10FB40002020015521460448FFF77EFF10BD418863
:10FB5000491C418010BD00009420002010B50748CA
:10FB60000068416A806A814203D300680449884280
:10FB700002D00120FEF7BAFF10BD0000B8F4FF1F4D
:10FB8000A52E5AE2024948600221417070470000E8
:10FB9000B8F4FF1FF7B51546394A00200446374927
:10FBA000128802E08300CC50401C9042FAD33548C2
:10FBB000302201883448FCF79DFE3448012100883A
:10FBC000C90780B24218324801683248FCF792FEF9
:10FBD00031480822018831480068FCF78BFE304F1D
:10FBE000FF26FE707C842F4A00213846FFF748FD2F
:10FBF0002D480421017044602C480170C4600461E8
:10FC00008482786A2030F8F79FFA29482A490760E9
:10FC1000022078702748047044700978C170FFF79B
:10FC200051FD2648016A320411430162C169026A2A
:10FC30005202920E92061143C161FEF77FFF2049E6
:10FC40000028086012DB82081E49920051180A68D9
:10FC50008307DB0E9E4032430A60C206D20E0121AA
:10FC600091404011184A80008018016000232A4604
:10FC70000199009800F084F8FEBD00007C2200206D
:10FC8000CE410100E4410100F4200020D0410100F8
:10FC9000E8410100C0210020EE410100CCF4FF1F2B
:10FCA000C420002039EB000094200020AC2000206C
:10FCB000B8F4FF1F58220020EC41010000ED00E0E5
:10FCC000B4F4FF1F00E400E000E100E010B50B48D1
:10FCD0000121026851700068FFF7D4FEFFF7CAFBEC
:10FCE00007480168491C0160FFF7C6FB00F028F8CF
:10FCF0000448FFF7B0FCFFF745FF10BDB8F4FF1F45
:10FD0000C0F4FF1F942000200148006870470000E5
:10FD1000C0F4FF1F074C084F2089BC4680B200DFAB
:10FD2000064FBC4600DF61680029F9D000208847F3
:10FD3000F6E70000A4F4FF1F15F700002DF7000000
:10FD400070B50D4D2868002815D0A8880B4E401EB0
:10FD5000A8800AE0E088FEF708FFA088A880206855
:10FD6000286021463068FFF763FCA888002802D18C
:10FD70002C68002CEED170BDC4F4FF1FCCF4FF1F23
:10FD8000FFB5080681B01E4617460C46000E00D18E
:10FD90004C1C1648FFF742FB051E25D02002000C24
:10FDA000AF626884EE61E1B22846019AFFF768FC11
:10FDB000104801240E49028806E0A000401880384F
:10FDC000C06F002803D0641C9442F6D90024A00020
:10FDD00040188038C567EC702846FFF789FB064855
:10FDE000006820300470204605B0F0BDF4200020EB
:10FDF0007C220020CE410100B8F4FF1F02480068B9
:10FE0000002800D0C0787047B8F4FF1F704700008A
:10FE1000F8B500250024FEF721F9064605215848CB
:10FE2000F8F7F9FB21215748F8F7F3FB2121564851
:10FE3000F8F7EFFB09215548F8F7EDFB052150488D
:10FE4000F8F7E9FB00BF00BF0AE0514BAA00995840
:10FE50004C4A101902F036FA0019C4B2681CC5B237
:10FE6000042DF2DB00222046611CCCB245490A5425
:10FE7000002400250AE0474BAA009958424A10196D
:10FE800002F020FA0019C4B2681CC5B2042DF2DBDE
:10FE900000222146601CC4B23B48425400243B4926
:10FEA00008193D49096802F00DFA0019C4B220464C
:10FEB000611CCCB2354900220A54FEF7BDF8074652
:10FEC000042239462E48F8F7F3FA2D49002008712C
:10FED00000243104080FFEF775F9014622462F4829
:10FEE000641C81543105080FFEF76CF90146224667
:10FEF0002A48641C8154FCF7B5FF012803D0FDF7A4
:10FF0000E7FB00280CD13111082211430807000F2C
:10FF1000FEF758F92146621CD4B2204A505408E03A
:10FF20003106080FFEF74EF92146621CD4B21B4A77
:10FF300050543007000FFEF745F92146621CD4B239
:10FF4000164A505400222046611CCCB213490A5470
:10FF50000024302221461248641C42543222214699
:10FF6000641C425435222146641C425434222146EA
:10FF7000641C425400222146641C4254F8BD000017
:10FF80003CF0FF1F6AF6FF1F8BF6FF1FACF6FF1F4A
:10FF90000CF6FF1F1CF6FF1F28F0FF1F41F0FF1F8C
:10FFA00046F0FF1FF1B5394DA869416900988847AF
:10FFB0000746A8698169009888470446002F07D042
:10FFC000002C05D00126B602B74209D8012008E06E
:10FFD000FF2232322EA10020FCF7CEFC0220F8BD19
:10FFE0000020FF2237322AA1FCF7C6FC39463046F2
:10FFF000F8F72CFB002909D00020FF22383224A179
:020000040001F9
:10000000FCF7BAFCBC4203D3012002E00120F4E774
:100010000020FF2239321EA1FCF7AEFC39462046F3
:10002000F8F714FB00291AD00020FF223A3218A159
:10003000FCF7A2FC21460098F8F708FB0098401A4C
:10004000E8602C616860B44200D33446AC60A969B2
:10005000096A002905D0884704000BD101E001207E
:10006000E3E7287800280AD0A869C168E8688847CB
:10007000040004D0A869406880472046F8BDFF22EC
:100080001048A968F8F7A0FA0020F8BDBCF0FF1FDF
:100090002E2E5C2E2E5C2E2E5C736F757263655C4B
:1000A0006461706C696E6B5C647261672D6E2D6447
:1000B000726F705C666C6173685F6D616E616765BD
:1000C000722E630050F8FF1F70B500250024002633
:1000D0001148F8F767F9C6B27000801CC2B2214619
:1000E0000E48641C425403222146641C425400BF43
:1000F0000EE00948611C425D2046CCB207490A5413
:1001000000222046611CCCB204490A54681CC5B2C6
:10011000B542EEDB70BD00002CF6FF1FB5F6FF1FE9
:1001200010B531210948F8F776FA09490748F8F778
:100130005BF908490548F8F757F907490348F8F704
:1001400053F906490148F8F74FF910BD2CF6FF1F87
:100150003CF0FF1F41F0FF1F6AF6FF1FACF6FF1FC8
:1001600010B50A4C2078002808D000F089F86068A3
:10017000C168074888470021217010BDC02205A131
:100180000020FCF7F9FB022010BD00007CF0FF1FEF
:100190001CF7FF1F2E2E5C2E2E5C2E2E5C736F75AF
:1001A0007263655C6461706C696E6B5C64726167DC
:1001B0002D6E2D64726F705C66696C655F7374720E
:1001C00065616D2E6300000070B5134C0546207804
:1001D000002801D0852202E0022D06D38B220FA138
:1001E0000020FCF7C9FB022070BDFEF731FCFF21A7
:1001F000A06005311648F8F70EFA01200649207074
:1002000028010C3140186060416811488847002877
:10021000EAD00321217070BD7CF0FF1F2E2E5C2ED2
:100220002E5C2E2E5C736F757263655C6461706CFE
:10023000696E6B5C647261672D6E2D64726F705CA9
:1002400066696C655F73747265616D2E6300000092
:100250001CF7FF1FF8B5094D0E4607460024200184
:100260002A58314638469047002801D02046F8BD2C
:10027000641CE4B2022CF2D30320F8BD88F0FF1F07
:1002800010B5FEF7E5FB06498968884201D10120D7
:1002900000E00020622203A1FCF76EFB10BD00000D
:1002A0007CF0FF1F2E2E5C2E2E5C2E2E5C736F7545
:1002B0007263655C6461706C696E6B5C64726167CB
:1002C0002D6E2D64726F705C66696C655F737472FD
:1002D00065616D2E63000000014610B508310322F0
:1002E0000C4608A0F8F794F8002807D0032221460E
:1002F00005A0F8F78DF8002801D0032010BD0120DB
:1003000010BD000042494E004845580070B5154DDB
:10031000064628780C46012806D0A42212A1002007
:10032000FCF72AFB022070BDFFF7AAFF686822468F
:1003300083683146194898470446132807D0142C7F
:1003400007D0002C05D003202870204670BD022065
:10035000FAE72878012800D00020B22202A1FCF799
:100360000BFBF2E77CF0FF1F2E2E5C2E2E5C2E2E58
:100370005C736F757263655C6461706C696E6B5CF5
:10038000647261672D6E2D64726F705C66696C6556
:100390005F73747265616D2E630000001CF7FF1FB0
:1003A00010B51E21002000F063FD002800D00120C0
:1003B00010BD0000F0B593B00F4604461E4615462A
:1003C00044216846F8F727F9189800950290199883
:1003D00003900196201DF8F720F909902046083077
:1003E000F8F71BF90D902046F8F717F90E90012049
:1003F000000610900F97684600F0F0FC00281BD014
:10040000114D124E002411A9304600F0C7F9002802
:1004100011D01198800311D56946002000F012F91F
:10042000002809D00A49304600F078FD002803D0A2
:100430000098002806D0002013B0F0BD641CAC4228
:10044000E1D3F8E70120F7E740420F00F0ED00E0CC
:1004500003005FA010B5044600F0CAFF002801D1D8
:10046000200E000610BD000010B5F8F709FF09487E
:1004700020214160402444600222426043690B43D2
:100480004361416921434161416911434161012057
:1004900010BD000080F00F40F8B50020411E009014
:1004A00035486426016004274160002412E0002CD6
:1004B00010D00121002000F0DBFC012000F048FA00
:1004C0000220FEF769FA002000F042FA0220FEF74F
:1004D00063FAEAE7FFF7C8FF28480068002803D05E
:1004E0008068002800D08047F9F736F900283CD012
:1004F000FFF756FF002838D00021082000F0B8FC94
:10050000002832D005210907042000F0B1FC0028A2
:100510002BD000250BE06946042000F0E9F8002804
:1005200021D0052000994007884302D06D1CB542B8
:10053000F1DBB54219D0012C17D01149042000F08D
:1005400097FC002811D00D480068002803D00069EE
:10055000002800D080470021082000F089FC0028F6
:1005600003D00120F8BD0124E3E77F1E01247FB200
:10057000002F9CDC0020F8BD64F0FF1FD0F4FF1FAB
:10058000000F0050074841692022914341614169B1
:10059000402291434161416902229143416101201E
:1005A0007047000080F00F40F8B50D460446002A61
:1005B0002CD096081649002000F052FB002826D0C7
:1005C0000527042221466846FDF740FF6946384664
:1005D00000F036FB012819D10F270021384600F022
:1005E0002FFB012812D10024761E07E02946384649
:1005F00000F026FB012809D1641C2D1DB442F5D35F
:100600000E20294600F01CFB012800D00020F8BD78
:100610005200002338B50D4604460949002000F079
:100620001FFB00280BD06946204600F033F8002855
:1006300005D0A007C10E0098C8402870012038BD21
:1006400050000023F8B50E460146002464251048EA
:1006500000F064FC002810D00D4F3F1F3146384693
:1006600000F09CF8002808D03068C00302D4641C55
:10067000AC42F3DBAC4201D10020F8BD0448314666
:10068000001D00F08BF80028F7D00120F8BD000015
:10069000F4ED00E01CB50C460146042201A8FDF76C
:1006A000D5FE052001A900F0CBFA01281ED10F20AC
:1006B000694600F0C5FA012818D10E20694600F0FD
:1006C000BFFA00216A462160D1780906216092783C
:1006D000120411436A4621605278120211436A469D
:1006E0002160127811432160012800D000201CBD38
:1006F00038B50C460C2108406946801C00F0A0FA71
:1007000000216A462160D17809062160927812049E
:1007100011436A4621605278120211436A462160F1
:10072000127811432160012800D0002038BDF8B5AF
:1007300014460F46054608E039462846FFF76AFF8B
:10074000002829D0641E6D1C7F1C002C23D0A80714
:10075000F2D112E0A9050120890D8002461AB442A7
:1007600001D2A608B600324639462846FFF71CFFDC
:10077000002811D0AD19BF19A41B032CEAD808E03A
:1007800039462846FFF746FF002805D0641E6D1C39
:100790007F1C002CF4D10120F8BD000070B50C4680
:1007A00005460749002000F05BFA002806D02146E4
:1007B0002846FFF76FFF002800D0012070BD000021
:1007C000520000231CB500206A46FF211154401C32
:1007D000C0B20828FAD311463320F9F7D7FA01201E
:1007E0001CBD000001490870704700005CF0FF1F4D
:1007F00001494860704700005CF0FF1FFEB50646E7
:100800000224FFF731FE4E4D3300FCF731F80504AA
:10081000170873769600012000F09AF88BE001200B
:1008200000F096F80220FEF7B7F8002000F090F8EC
:100830000220FEF7B1F8FFF7A5FE7CE0FFF72CFEE3
:10084000002879D03F4E2846314600F067FB00284B
:100850003BD069462846FFF7A1FF00286CD00098DE
:100860008003F6D5384E012401A93046FFF796FFE4
:10087000002861D0019901200143304600F04EFB71
:10088000002859D02E4F6946E43F3846FFF786FFCF
:10089000002851D00098790D08402C49411838465D
:1008A00000F03CFB002847D00A20FEF775F86946A7
:1008B0002846FFF773FF00283ED000988003F6D546
:1008C000002C13D03046019931E0641E64B2002C34
:1008D00033DD012000F03CF80220FEF75DF8002037
:1008E00000F036F80220FEF757F8ACE71448002174
:1008F0000C301CE01349C91E18E0F8F72DFF002842
:100900001AD01E21002000F0B3FA002814D00021D4
:10091000082000F0ADFA00280ED0052109070420B8
:1009200000F0A6FA002807D00649891E284600F0E4
:10093000F5FA002800D00120FEBD0020FEBD000019
:10094000F0ED00E003005FA0B00104400400FA05F0
:1009500007490968002903D0C969002900D0084760
:1009600002220449002801D08A6070474A6070471B
:10097000D0F4FF1F80F00F40F8B50224054606288A
:1009800001D0FFF771FD4E494E4E4F1C2B00FBF777
:100990006FFF080516095C5E758C93950120FFF7C3
:1009A000D7FF89E00120FFF7D3FF0220FDF7F4FF16
:1009B0000020FFF7CDFF0220FDF7EEFF7AE0FFF702
:1009C0006BFD002879D0404D287801280BD00FE02E
:1009D000641E64B2002C71DD0120FFF7B9FF022014
:1009E000FDF7DAFF0020FFF7B3FF0220FDF7D4FF89
:1009F0003946304600F092FA0028E9D0314C012106
:100A00000C34204600F08AFA002856D028780028B6
:100A100005D10120FFF79CFF0220FDF7BDFF00205C
:100A2000FFF796FF0220FDF7B7FF69463046FFF754
:100A3000B5FE002841D000988003F6D5002120465D
:100A400000F06CFA002838D036E03046F8E7F8F7C6
:100A500083FE002831D0FFF7A3FC00282DD0002111
:100A6000082000F005FA002827D0052109070420F6
:100A700000F0FEF9002820D03946E6E7FFF70CFD2C
:100A800000281AD00E493046C91C00F047FA002849
:100A900013D069463046FFF781FE00280DD000983C
:100AA0008003F6D508E008E008E0304600F036FAAA
:100AB000002802D0FFF766FD0120F8BD0020F8BD38
:100AC00000005FA0F0ED00E05CF0FF1FF8B502242D
:100AD0000546062801D0FFF7C7FC5549554ECF1CE7
:100AE0002B00FBF7C5FE080516096A6C849AA1A3C2
:100AF0000120FFF72DFF97E00120FFF729FF0220DB
:100B0000FDF74AFF0020FFF723FF0220FDF744FF17
:100B100088E0FFF7C1FC00287DD00FE0641E64B2BE
:100B2000002C79DD0120FFF713FF0220FDF734FFD1
:100B30000020FFF70DFF0220FDF72EFF394630465B
:100B400000F0ECF90028E9D069463046FFF726FEB0
:100B500000286AD000988003F6D5364C01210C3469
:100B6000204600F0DBF900285FD0324D6946E43DB5
:100B70002846FFF713FE002857D00098610D084063
:100B80002D4941182D4840680143284600F0C6F918
:100B900000284AD00220FDF7FFFE69463046FFF7E5
:100BA000FDFD002841D000988003F6D500212046A5
:100BB00000F0B4F9002838D036E03046F8E7F8F70E
:100BC000CBFD002831D0FFF7EBFB00282DD0002112
:100BD000082000F04DF9002827D00521090704203E
:100BE00000F046F9002820D01149491CE5E7FFF73D
:100BF00053FC002819D03946304600F08FF9002800
:100C000013D069463046FFF7C9FD00280DD0009883
:100C10008003F6D508E008E008E0304600F07EF9F1
:100C2000002802D0FFF7AEFC0120F8BD0020F8BD7F
:100C300000005FA0F0ED00E00000FA055CF0FF1F8F
:100C400070B50D460646002429463046F8F714FED6
:100C5000022803D1641CE4B2642CF5D370BD0000FB
:100C600038B50D460446FFF7F5FB2246F0210A4051
:100C700010430146082000F0FBF8002806D0002CA5
:100C800006D10E484168A94201D1012038BD456016
:100C90000C200440042229466846641CFDF7D6FB5C
:100CA00069462046FFF7CCFF012805D10E20002120
:100CB000FFF7C6FF0128E9D0002038BD64F0FF1F10
:100CC000F8B50D460446002A25D0960813490020A1
:100CD000FFF7C6FF00281FD00527042221466846DB
:100CE000FDF7B4FB69463846FFF7AAFF012812D189
:100CF0000D27002407E029463846FFF7A1FF012809
:100D000009D1641C2D1DB442F5D30E200021FFF73C
:100D100097FF012800D00020F8BD000052000023FA
:100D200070B50C46054608490020FFF799FF0028DA
:100D300009D0A807C00E21468140284600F02EF8B1
:100D4000002800D0012070BD5000002373B5064676
:100D5000002464251048019900F0E0F8002815D01F
:100D600001200004314601430B48001F00F0D6F873
:100D700000280BD0084E083E01A93046FFF70EFDB3
:100D8000002803D00198C00301D501207CBD641C5C
:100D9000AC42F1DB00207CBDF8ED00E038B50C463C
:100DA000014604226846FDF751FB05206946FFF71E
:100DB00047FF012810D1042221466846FDF746FB73
:100DC0000D206946FFF73CFF012805D10E200021C8
:100DD000FFF736FF012800D0002038BD38B50546A2
:100DE0000021082000F044F800283AD00024A00098
:100DF00029582046FFF7AAFF002832D0641C042C93
:100E0000F5D30920696AFFF7A1FF002829D00D2436
:100E1000A00029582046FFF799FF002821D0641C24
:100E2000102CF5D31020296CFFF790FF002818D064
:100E30000E4C0D49204600F071F8002811D00A49E7
:100E40002046891E00F06AF800280AD0694604206E
:100E5000FFF74EFC002804D00098A021084201D0E2
:100E6000002038BD012038BD0B005FA0F0ED00E090
:100E7000F8B50E4F04460E46082802D13868B04235
:100E800011D00C202546054004226846FDF7DEFA05
:100E900069462846FFF7D4FE012801D00020F8BD9E
:100EA000082C00D13E600120F8BD000064F0FF1F57
:100EB000F8B514460D46064608E029783046FFF797
:100EC0002FFF002829D0641E6D1C761C002C23D017
:100ED000B007F2D112E0B1050120890D8002471A56
:100EE000BC4201D2A708BF003A4629463046FFF768
:100EF000E7FE002811D0F619ED19E41B032CEAD8FF
:100F000008E029783046FFF70BFF002805D0641E63
:100F10006D1C761C002CF4D10120F8BD70B50C4678
:100F2000054607490020FFF79BFE002806D0214612
:100F30002846FFF733FF002800D0012070BD0000D5
:100F40005200002310B5FDF783FD06494968884229
:100F500001D1012000E00020FF22693202A1FBF74D
:100F60000BFD10BDFCF0FF1F2E2E5C2E2E5C2E2ED6
:100F70005C736F757263655C6461706C696E6B5CE9
:100F8000647261672D6E2D64726F705C7666735F3C
:100F90006D616E616765722E6300000010B50348D5
:100FA0000021C068FDF712FD10BD0000FCF0FF1F1E
:100FB00010B50248C068FDF71FFD10BDFCF0FF1F13
:100FC00002480078012800D0002070476CF0FF1F15
:100FD00002480078012800D000207047D8F0FF1F99
:100FE000FEB521480546F7F718FB002839D0002642
:100FF00004460C341CE0384600F0AAF900282DD134
:101000000120FCF737FE060028D11848476838460B
:101010000830F7F702FB002100910B460A460191C8
:10102000014638461830FFF7C5F9002817D01434A8
:101030002046F7F7F2FA0700DDD1201DF7F7EDFAA9
:101040000028D8D12846F7F7E8FAFF30A130807899
:10105000002802D000F08AF806463046FEBD102077
:10106000FEBD0120FEBD0000183001006CF0FF1F26
:101070007CB505461748F7F7D0FA002828D016485F
:101080004468002C09D0284600F028F8014628467C
:10109000F7F7DCFA002919D101E002207CBD01201C
:1010A000FCF7E8FD0028F9D120460C30F7F7B5FA37
:1010B000002100910B460191014620462A46183036
:1010C000FFF778F9002801D000207CBD0F207CBDFF
:1010D00001207CBD183001006CF0FF1F70B5054683
:1010E0001448F7F79AFA061E18D030460830F7F77A
:1010F00094FA002815D0441E13D4301DF7F78DFA4A
:10110000E1004018F7F789FAA84208D8301DF7F730
:1011100084FAE100091D4018F7F77FFA70BD641EDC
:10112000EBD5FF227A3204A10020FBF725FC00203A
:1011300070BD0000183001002E2E5C2E2E5C2E2E6D
:101140005C736F757263655C6461706C696E6B5C17
:10115000696E746572666163655C746172676574FB
:101160005F666C6173682E630000000070B51848FC
:101170000446F7F752FA002827D0164D0020687071
:101180006860012000F040F9002805D02046F7F7FC
:1011900044FA04460C340AE0072070BD20460830AB
:1011A000F7F73BFAC00701D0AC600AE014342046E0
:1011B000F7F733FA0028F1D1201DF7F72EFA0028AF
:1011C000ECD101202870002070BD012070BD00000E
:1011D000183001006CF0FF1FF7B584B015464E487B
:1011E000F7F71BFA002870D04C484768002F12D040
:1011F0004B480068002808D04369002B05D02A46D8
:10120000059904989847012808D00220FCF732FD80
:10121000002801D155E0022007B0F0BD0D20FBE70A
:1012200038463430F7F7F9F9A84201D92C4600E0E6
:101230000446384624300290F7F7EFF92246059924
:10124000FFF736FE002858D00298F7F7E6F900902D
:1012500038461030F7F7E1F90146384600261830D5
:1012600023460196049A0390FFF7A4F800282DD096
:10127000FBF732FD00281DD0384614300090F7F7F8
:10128000CCF9002843D00320FCF7F4FC0028C3D19C
:101290000298F7F7C2F901900098F7F7BEF90199A3
:1012A0000091014623460196049A0398FFF782F8BD
:1012B000002820D0049800190490059800192D1BCF
:1012C0000590002DACD10020A6E723E01120A3E774
:1012D000102C01D2264600E01026324669460498BA
:1012E000FFF725FA002808D0324669460598F7F737
:1012F0002BF8002803D012208EE70A208CE70498F0
:10130000AD1B8019049005988019A41B0590002C32
:10131000D7D0DDE701207FE7183001006CF0FF1F18
:10132000D0F4FF1F70B505460848F7F776F9002896
:101330000BD0FF2401342846FFF7D0FEA04203D291
:101340002846FFF7CBFE0446204670BD183001004A
:10135000F8B5FCF7A1FE04001FD0124D6868A0424A
:1013600019D00020FCF786FC002815D120462C302F
:10137000F7F753F9074620463030F7F74EF906469F
:1013800020462830F7F749F93A463146FFF790FDF5
:10139000002804D06C600020F8BD0920F8BD0820AA
:1013A000F8BD00006CF0FF1F10B50F48F7F735F9D6
:1013B000002817D00020FCF75DFC002811D1FBF7B6
:1013C00083FC002801D0022000E0012000F01CF87E
:1013D000072000F019F8054900200870FFF7D2F83F
:1013E000002010BD012010BD183001006CF0FF1F5F
:1013F00004480068002802D0806A002800D100203C
:1014000070470000D0F4FF1F70B505461648F7F787
:1014100004F9010001D02846884714480468002CCC
:101420001FD0A169002902D02846884770BDA07846
:10143000012803D0022805D0012070BD2846FFF7FF
:101440009BFA70BD0848001DF7F7E7F8002802D1A5
:101450006068002801D0FFF7CBF92846FFF736FB7C
:1014600070BD002070BD00007A300100D0F4FF1F75
:10147000884203D3904201D8012070470020704772
:1014800070B5094C0221E068FDF7BEFAA06803219F
:101490000546F7F7DBF86D1CA560002903D1012193
:1014A000E068FDF7B1FA70BD4CF0FF1FF8B51B4CBA
:1014B0001546E0780E46002805D0194A19A10020EB
:1014C000FBF75AFAF8BDE8051ED00020144A15A112
:1014D000121DFBF751FAB1226078920011A1FBF7BF
:1014E0004BFA29463046FEF711FF00270126132844
:1014F0000CD014280FD02771084920394A69521995
:101500004A6100F0CDF8F8BD0120DFE7FEF728FEC4
:101510006770E67000E000202671EDE7BC02002055
:10152000BF0200002E2E5C2E2E5C2E2E5C736F757B
:101530007263655C6461706C696E6B5C6472616738
:101540002D6E2D64726F705C7666735F6D616E6177
:101550006765722E63000000F8B51A4C0746607884
:101560000D46002812D00020A122920016A1FBF700
:1015700003FA681C00D00120204A13A1FBF7FCF9F4
:10158000104E203E7068401C02D002E00120EBE7C4
:101590007560E079032800D1E7717068A84202D134
:1015A000E079B84201D0032008E03846FEF70CFE8F
:1015B000002803D10121F5606170A17000F070F87E
:1015C000F8BD0000BC0200202E2E5C2E2E5C2E2EBC
:1015D0005C736F757263655C6461706C696E6B5C83
:1015E000647261672D6E2D64726F705C7666735FD6
:1015F0006D616E616765722E6300000085020000F8
:1016000070B5194C2578032D05D02546203D2E6850
:10161000002E07D007E08D22920014A10020FBF7D6
:10162000ABF970BD2860A868401C00D1A960E079C2
:10163000032800D1E371A869904206D9E869904275
:1016400003D9002A01D003200BE0481C02D0A8686F
:101650008842F8D1032B02D0E0799842F3D10020E0
:10166000AA6100F01DF870BDBC0200202E2E5C2E79
:101670002E5C2E2E5C736F757263655C6461706C9A
:10168000696E6B5C647261672D6E2D64726F705C45
:101690007666735F6D616E616765722E6300000030
:1016A000FEB50546132803D0142D01D0012000E01B
:1016B0000020B922920045A1FBF75EF9504C20783A
:1016C000032810D02246203A1168002912D0D3698D
:1016D000906983420ED300280CD0936850689842DA
:1016E00008D1012007E05D22D20038A10020FBF7DD
:1016F00043F9FEBD00206071A3790193002902D156
:10170000E179032901D0012100E0002100910028A6
:1017100004D02179002901D0012600E00026E178DB
:10172000002903D0002801D0012000E00020029011
:1017300010690027401C13D0314820384068401CF5
:1017400000D001202F4A21A1FBF716F92C482038A0
:10175000426801694069891A4902884200D9012713
:101760000320002D01D020701DE0019900290AD02E
:10177000002F01D00625F6E700990029F3D0002EAE
:10178000F1D10425EFE702990029ECD1002E01D018
:10179000022003E00098002802D00120207011E010
:1017A000207803280BD16078002806D0FEF7D8FCFB
:1017B00000216170002D00D1054613480570019885
:1017C000002896D101F066F8FEBD00002E2E5C2E9A
:1017D0002E5C2E2E5C736F757263655C6461706C39
:1017E000696E6B5C647261672D6E2D64726F705CE4
:1017F0007666735F6D616E616765722E63000000CF
:10180000BC02002006030000FCF0FF1F10B50D20F5
:10181000FBF748F81348826BC1140A438263426B9A
:101820000A434263104CE078F3210840E070E0780E
:101830005F210840E070FBF707FA0D480B49C160D3
:10184000C91E0161E0780C210843E070E078202196
:101850000843E0700D20FBF719F80D20FBF732F874
:10186000012010BD0080044000B0064003030000CA
:1018700000B004400A4610B501460248FBF7BAF929
:1018800010BD00009810002010B50D20FBF70AF8DD
:101890000548C1784906490EC170FBF7D5F90D20FE
:1018A000FBF710F8012010BD00B00640F8B5064661
:1018B00000252F460D20FAF7F5FF1E4CE0785F213A
:1018C0000840E070E078F3210840E070FBF7BCF9D5
:1018D00071790020012902D0022903D004E00125FA
:1018E0002F4600E00125012000016900084338432C
:1018F000A0703068010110480068F6F7A7FE217853
:10190000400849094901C204D20E1143217061788F
:101910006070E0780C210843E0700D20FAF7B6FF04
:101920000D20FAF7CFFFE07820210843E070012076
:10193000F8BD000000B00640D8F2FF1F70B50A469F
:1019400001460C48FBF76BF90546EFF31080C4071E
:10195000E40F72B60748FBF7B4F8002804D0064835
:10196000C17880221143C170002C00D162B6284694
:1019700070BD0000880E002000B0064010B502487F
:10198000FBF78EF810BD0000880E002010B50F4C3C
:101990002078002807D000202070FAF767FF002881
:1019A00008D01E2010BD832209A10020FAF7E4FF11
:1019B000022010BD6078002803D1FBF712FC00283C
:1019C00001D0002010BD242010BD0000D8F0FF1F62
:1019D0002E2E5C2E2E5C2E2E5C736F757263655CF2
:1019E0006461706C696E6B5C647261672D6E2D64EE
:1019F000726F705C6961705F666C6173685F696E5D
:101A000074662E6300000000F8B50F460446F6F732
:101A100000FE20468DA100F07BFC0546601998A1D0
:101A200000F076FC4519601999A100F071FC451988
:101A300060199BA100F06CFC4519FBF745F90028E3
:101A400001D09BA100E09BA1601900F061FC451949
:101A5000601999A100F05CFC4519601997A100F08C
:101A600057FC4519FBF738F9002801D090A100E098
:101A700090A1601900F04CFC451960198EA100F08E
:101A800047FC4519601993A100F042FC4519FBF78A
:101A90002BF9002801D086A100E086A1601900F092
:101AA00037FC4519601984A100F032FC4519FBF799
:101AB00098FB002801D08DA600E08FA6601991A1A7
:101AC00000F026FC45196019314600F021FC45194B
:101AD000601979A100F01CFC45196019314600F02D
:101AE00017FC451960198BA100F012FC4519FBF792
:101AF00078FB002815D1FCF7C9FB002811D060192C
:101B000088A100F005FC4519FCF7D2FB01466019DD
:101B1000042200F02CFC4519601967A100F0F8FBC5
:101B20004519FBF760FB002815D1FCF7DFFB002807
:101B300011D0601981A100F0EBFB4519FCF7EAFB1D
:101B400001466019042200F012FC451960195AA1DF
:101B500000F0DEFB451960197DA100F0D9FB4519A5
:101B600060197EA100F0D4FB4519601952A100F064
:101B7000CFFB4519601984A100F0CAFB4519601913
:101B8000012100F0CEFB451960194BA100F0C0FB0C
:101B90004519601980A100F0BBFB4519601983A1AC
:101BA00000F0B6FB4519601981A100F0B1FB4519A1
:101BB000601981A100F0ACFB4519601980A100F00B
:101BC000A7FB451960193CA100F0A2FB4519FCF7E1
:101BD0005DFB002810D060197CA100F099FB45192D
:101BE000FCF770FB0146601900F06CFB45196019A9
:101BF00031A100F08DFB4519601979A100F088FB37
:101C00004519FCF765FB0146601900F05BFB4519BF
:101C1000601929A100F07CFB4519601975A100F03D
:101C200077FB784945196019496800F07AFB451936
:101C3000601921A100F06CFB4019201872A100F07E
:101C400067FB39462046FBF7C9FBF8BD232044411A
:101C5000504C696E6B204669726D77617265202DFC
:101C6000207365652068747470733A2F2F6D6265F8
:101C7000642E636F6D2F6461706C696E6B0D0A006A
:101C8000556E697175652049443A2040550D0A002A
:101C90004849432049443A2040440D0A00000000CE
:101CA0004175746F2052657365743A20000000001E
:101CB00031000000300000000D0A00004175746F13
:101CC0006D6174696F6E20616C6C6F7765643A202A
:101CD000000000004F766572666C6F772064657453
:101CE000656374696F6E3A2000000000426F6F7484
:101CF0006C6F616465720000496E74657266616341
:101D0000650000004461706C696E6B204D6F646506
:101D10003A2000002056657273696F6E3A20405673
:101D20000D0A0000426F6F746C6F6164657220561B
:101D3000657273696F6E3A2000000000496E746529
:101D400072666163652056657273696F6E3A200032
:101D5000476974205348413A2000000031366365DA
:101D60003165386438393133613233666461313515
:101D700031396165386431336263333363326437D8
:101D800064663563000000004C6F63616C204D6F2A
:101D900064733A200000000055534220496E746578
:101DA0007266616365733A20000000004D53440081
:101DB0002C204344430000002C20484944000000EC
:101DC0002C2057656255534200000000426F6F742B
:101DD0006C6F61646572204352433A203078000092
:101DE000496E74657266616365204352433A2030E0
:101DF0007800000052656D6F756E7420636F756EAC
:101E0000743A20000CF1FF1F55524C3A2040520DFD
:101E10000A00000010B5064C044860600020608095
:101E20000448F7F7BBFA0120207010BDF21400201F
:101E300018F5FF1F38230020F0B54BA30ECB9DB043
:101E40006D460EC5474F0024384609226946F6F70D
:101E50002FFB0925FBF706F8464E012873D0FBF748
:101E600037FC00286FD074712046019001247D1941
:101E7000182241A102A8F6F72BFA172202A9284638
:101E8000F6F716FB0198A870202500F0A7F934702A
:101E90002746641C334974704919009144223C4917
:101EA0000CA8641CF6F714FA42220CA90098F6F765
:101EB000FFFA0099781C8F70009942358F721F319C
:101EC000CF7008718873F8F769FA26493471491997
:101ED0000091671C20222FA102A8F6F7F9F9202211
:101EE00002A90098F6F7E4FA009920358C7000F00A
:101EF00005F9B7712FA10EC91A4803924019029132
:101F00007C1C04930090092202A9F6F7D1FA0098EC
:101F100009358770174818220C3087731148B47040
:101F2000451927A102A8F6F7D3F9172202A92846D6
:101F3000F6F7BEFA0F48AC70B6300471FFF76AFFCF
:101F40001DB0F0BDFFE730890649401E30810871A1
:101F50008B2088700022CA701F493A5408881738AD
:101F6000088094E7A81200200902A2000601008060
:101F7000FA000000DCF2FF1F09040000020806500E
:101F80000807058202400000070502024000000029
:101F90008C41010009040000020300000609210031
:101FA000010001222100070581034000010705010E
:101FB000034000010904000000FF030007000000C7
:101FC0000904000002FF00000907050502400000A7
:101FD0000705850240000000E6F2FF1F0248407836
:101FE000002800D00120704760F5FF1F10B5F8F7FA
:101FF0000FFB10BD002070477CB51C46154601281C
:102000001ED1002C01D0012C1AD101AA69460D481D
:10201000F7F7A4F900280ED0019A402A05DD4F22D7
:1020200009A10020FAF7A8FC0AE028460099F6F773
:102030003FFA40207CBD012C02D10D4901200870DF
:1020400000207CBDC02400202E2E5C2E2E5C2E2E67
:102050005C736F757263655C7573625C6869645C00
:10206000757362645F757365725F6869642E63007F
:10207000E0F5FF1FF8B507461A4816460088824269
:1020800001DD0020F8BD184800780028FAD0174C70
:102090000122E26001E0002814D06288002AFAD10F
:1020A000134D32462F70681CF6F702FA2046656120
:1020B0000024848046800F490978012908D86D1CC6
:1020C000456108E00020E0606061A0806080D8E7A2
:1020D0004188491C41800020F8F7C0FD0648C455DE
:1020E0000120F8BD7E3F010061F5FF1F84F5FF1F51
:1020F000B01300207C3F010080F4FF1F10B503499E
:10210000012008700248F7F749F910BDE0F5FF1FFC
:10211000C02400200178832902D14078002801D012
:1021200000207047012070477047000038B5012437
:102130001D461146022814D1002D12D00878072818
:102140000CD06B462A461148F7F7DAF8002813D06E
:102150000098FFF7DFFF012804D004E00C490120BC
:10216000087038BD00240B4D2878002809D0FCF7F2
:102170002FF80020287004E0852207A10020FAF73C
:10218000FBFB2046FCF760FA38BD0000C0240020AD
:1021900000F0FF1FE0F5FF1F2E2E5C2E2E5C2E2E72
:1021A0005C736F757263655C7573625C6869645CAF
:1021B000757362645F757365725F6869642E63002E
:1021C00010B505490020C870FFF736FEF9F7B2FEDA
:1021D000F9F722F810BD000060F5FF1F10B5FCF7FD
:1021E00037FC074C60600020FCF7FAFBE060FAF770
:1021F000E7FB00206070A0700249A060086010BD7D
:10220000FCF0FF1FACF5FF1F70B514460D460646E7
:10221000FEF798FE064B1868002807D00120FCF74F
:102220001BFA22462946304600F0BEFB70BD000076
:10223000ACF5FF1F70470000F8B515460E4607467F
:10224000FEF780FE0D480068002816D00C490020DB
:102250000C4C8860207803280FD00120FCF7FCF993
:102260002A463146384600F031FD2078032804D054
:102270002A4631463846FBF7B1F9F8BDACF5FF1FE9
:10228000FCF0FF1FBC0200200548074A0178054802
:10229000C180002101704170C1608260016170479E
:1022A0006E3F010060F5FF1F0100010010B5EFF364
:1022B0001080C407E40F72B6FAF78AFD002C00D133
:1022C00062B610BD70B50D460446090E00F014F854
:1022D00006462802010EA01900F00EF886192804FF
:1022E000010EA01900F008F88619E9B2A01900F053
:1022F00003F8801970BD00000B09044A0907D35C7C
:102300000370090F515C4170022070475431010085
:102310000346002001E01A54401C0A5C002AFAD14E
:102320007047F3B581B0074600242546029805E0C2
:102330000A21F6F78BF90021641C4D410028F7D1E2
:102340002046284301D101240025002609E00A2166
:102350000298F6F77BF9A21B3031521EB954761C55
:1023600002900020311BA841F1D32046FEBDF8B5F4
:1023700015460E460746FFF7D4FF0446A8420AD288
:10238000302229463846F6F71FF9281BC019314676
:10239000FFF7C7FF2846F8BDF1B5304882B00068A6
:1023A000002808D0016A002905D002988847002833
:1023B00000D00120FEBD2A480190F6F72EF9040056
:1023C0004AD000200425074600902A466846029914
:1023D000F6F76EF8D4340AE0201DF6F71EF902462F
:1023E00031460098FFF744F8012832D014342046D3
:1023F000F6F713F90600EFD1201DF6F70EF90028C5
:10240000EAD1002F28D024E00298002641190422A6
:102410006846F6F74DF80198F6F7FFF804460C34D5
:102420000AE0201DF6F7F9F8024639460098FFF752
:102430001FF801280CD014342046F6F7EEF80700F8
:10244000EFD1201DF6F7E9F80028EAD1002E03D0DD
:102450002D1D0C2DD8D9ACE70020FEBDD0F4FF1FF8
:10246000183001000C490968002903D0496A002985
:1024700000D0084701783A290AD1007A302809D0DB
:10248000322807D0332805D0342803D0352801D08E
:102490000020704701207047D0F4FF1FFFB583B0C4
:1024A0000398FBF7D7F8FF22973241A1FAF764FAB5
:1024B0004C480190417A007A090201434948C01E04
:1024C000407B414306984018401EF6F7BFF805468A
:1024D00006980027444E002819D00024681EF7688B
:1024E00000900AE0F168481C82B2404800F0EEFC1F
:1024F000F068401CF0600098641C8442F2D33C4AAF
:102500003A48F16800F0E2FCF068401CF060306985
:10251000202802D3FF22AC321FE04101354A401C83
:102520008C183061202234492046F5F7C1FF0B2278
:1025300020460399F5F7BCFF21461C310698F6F7B3
:102540007DF8380C2075000A6075A776380AE076A9
:10255000B168102908D3FF22BA3215A10020FAF77A
:102560000BFA002007B0F0BD08460C225043214A68
:10257000224BC03A1350224B87187B60049B002BE0
:1025800000D013500598002800D078600198491CAD
:10259000427A037A1002134A1843D21E527B5043E8
:1025A0006843B860B1603078401C30702046D9E78D
:1025B0002E2E5C2E2E5C2E2E5C736F757263655C06
:1025C0006461706C696E6B5C647261672D6E2D6402
:1025D000726F705C7669727475616C5F66732E637E
:1025E000000000000B05002014F1FF1F0807002069
:1025F000FFFF0000C80900208C350100E1F2000057
:1026000001300100C07A704710B51C30F6F705F8AC
:1026100010BD000010B50446FFF7F6FF002812D0E9
:10262000E07EA17E040209480C43017BC07A0902C6
:10263000014307484069F6F709F80449A41E497B9D
:102640006143081810BD0020C04310BD08050020DC
:1026500014F1FF1FC172704770B50F49087DCA7C25
:102660000402087BC97A050214430D43002C01D0F3
:102670006C430FE008482030F5F7CFFF002802D068
:102680006843044606E00024FF228B3203A1204663
:10269000FAF772F9204670BD080500202E2E5C2E38
:1026A0002E5C2E2E5C736F757263655C6461706C5A
:1026B000696E6B5C647261672D6E2D64726F705C05
:1026C0007669727475616C5F66732E63000000003A
:1026D000F3B501260F46760281B031464D48F5F735
:1026E0009AFF31464C48F5F796FF4C4C0025C02127
:1026F0004B48E560F5F78FFF49487100C030F5F7AA
:102700008AFF25612570A560464865616060324694
:1027100045494048F5F7DCFD3E4E307BF27A010238
:102720000120000411433818F61CF5F78FFF04460A
:10273000F71E797B3D484843A04208D9FF22583212
:102740003BA10020FAF718F97C7B38480BE045489C
:102750004143A14208D2FF225B3235A10020FAF7A3
:102760000BF97C7B3F4844432A4901200004203177
:10277000844204D33574280A7074204603E034740C
:10278000200A70740020F5F759FF797B2046F5F791
:102790005DFF3449000211394018040CFC823022DC
:1027A00031491F48F5F794FD60021D491B4C4861F3
:1027B000086204206561A06000200C224243521888
:1027C00092686369401CD21862610428F5D3254AD7
:1027D000294667321048E56000F078FBE168214A3D
:1027E000491C6E320C48E16000F070FBE068256126
:1027F0000B4D401C1C49E060C0352846202230317A
:10280000F5F756FE28460B220199F5F751FE0120F7
:102810002061FEBD080500200807002014F1FF1FFD
:10282000080900200DD500003C3301005A100000BB
:102830002E2E5C2E2E5C2E2E5C736F757263655C83
:102840006461706C696E6B5C647261672D6E2D647F
:10285000726F705C7669727475616C5F66732E63FB
:102860000000000091FF00003C35010010B5044657
:10287000FEF794FB0649002C07D08878002801D188
:1028800002208870FEF794FB10BD0020F9E70000DD
:10289000FCF0FF1F10B5FEF781FBFAF7F5F80028F2
:1028A00005D104484178022901D101218170FEF748
:1028B0007FFB10BDFCF0FF1F10B5FEF743FB014886
:1028C000007810BDFCF0FF1FF8B50446FEF73AFB98
:1028D000FEF764FBFAF7D8F8002810D0FCF708FDE3
:1028E000204A214B9168994201D209199160002830
:1028F00005D0947855785470012C05D102E0FEF78C
:1029000057FBF8BD0220907000269660FEF750FB42
:102910000127002D16D0012D14D0022D12D1134DF8
:102920002878032803D0AF710020FEF7B9FE28787D
:10293000032812D00020FF2211320DA1FAF71CF853
:1029400000F0F8F8174D002C09D0012C07D0022C0C
:10295000D7D1FAF735F82F60F8BD0120EBE72E60EC
:10296000F8BD0000FCF0FF1F60EA0000BC02002080
:102970002E2E5C2E2E5C2E2E5C736F757263655C42
:102980006461706C696E6B5C647261672D6E2D643E
:10299000726F705C7666735F6D616E616765722ED3
:1029A00063000000ACF5FF1FF7B582B00446154682
:1029B000002651020398F5F72CFE002031460C2228
:1029C00051430F4A8B189B685B0AC31800938442DB
:1029D0000CD39C420AD21F1BAF4200D32F46535840
:1029E000201A3A4603999847E419ED1B002D04D0AC
:1029F000761CF6B20098102EE0D305B0F0BD0000B2
:102A000008090020014948607047000014F1FF1FC9
:102A10001CB5304CE07F002802D020461F3000E07B
:102A20002DA001218906FFF753FE2E48FBF72CFB52
:102A30000346207D002802D02648143000E02AA05A
:102A400000222849FFF72AFD2A48FBF71DFB034611
:102A50000022284928A0FFF721FDFFF72DFF0028BD
:102A600008D02848FBF710FB03460022254926A082
:102A7000FFF714FD274B41219A1C2748FAF7B6F9B6
:102A800000280BD02548FBF7FFFA03460022234914
:102A90002348FFF703FD0021FFF7DCFD0020019034
:102AA0000120C0030090FAF79EFB002810D0FF22FF
:102AB000013200990198F5F747FC002808D1194820
:102AC000FBF7E2FA03460022164917A0FFF7E6FCDF
:102AD0001CBD0000083001004441504C494E4B20C1
:102AE0002020200041F200004D42454420202020BB
:102AF00048544D0085F1000044455441494C532051
:102B0000545854009DF100004641494C202020209B
:102B1000545854000CF1FF1FC404002055F000006D
:102B2000BB32010079F200004E4545445F424C2023
:102B30005458540010B5FAF754FB002805D0FFF79D
:102B4000BBFE002801D1F7F793F9FAF74CFB0028F8
:102B500009D0FAF79BF9002803D1FAF783F9012885
:102B600001D1F7F785F902484168491C416010BD61
:102B70000CF1FF1FF8B50C46074600F0A3F800283B
:102B800053D1FBF7BDFA002803D1FBF7B1FA0028B7
:102B900000D00120002803D1FAF79EF8002844D085
:102BA000022C42D0002C0BD0012C3ED10B223749F5
:102BB0003846F5F7C9FB002837D1FFF777FB62E00D
:102BC000012069460870851E384600F07DF800280F
:102BD00055D12E4E00240D36E00031580B223846D8
:102BE000F5F7B2FB002800D12546641C0C2CF3D36A
:102BF000681C0024002816D02B00F9F739FE0C07BA
:102C00000F40172224282A2E3034363AFAF7EBFAEE
:102C1000002834D00120FAF773F930E0E7221CA134
:102C20000020F9F7A9FE68460470F8BD244C20681E
:102C300000688047206800698047206840688047B6
:102C40001DE0012000E00020FAF7B0F917E00120B4
:102C500000E00020FAF7B4F911E0012000E00020C4
:102C6000FAF7B8F90BE0002000E00120FAF742F98A
:102C700005E0FF220A3206A10020F9F77DFE684632
:102C800000780028D1D0FFF705FEF8BDBB32010067
:102C90002E2E5C2E2E5C2E2E5C736F757263655C1F
:102CA0006461706C696E6B5C647261672D6E2D641B
:102CB000726F705C7666735F757365722E63000069
:102CC000503101000020704700207047F7B50446DE
:102CD000002682B0154630461CE00C2132464A439D
:102CE0000F4952189168490A4118009184420CD347
:102CF0008C420AD20F1BAF4200D32F465368201AD2
:102D00003A4603999847E419ED1B002D06D0761C2E
:102D10000098F6B2034989688E42DED305B0F0BD53
:102D20000809002014F1FF1FF7B5054604462035B9
:102D3000287C84B01646302801D3606B32E0302105
:102D40000F1AB74200D3174600193A460599F5F70E
:102D5000AFFB287CC019C1B22974302902D20020EF
:102D600007B0F0BD05980023C0190590F61B1A4660
:102D70002046FAF761FD00281FD002A90022009129
:102D800001AB1146FAF7B0FD0028E9D10198606364
:102D90002A7C2146FAF7BCFE0028E1D1297C606B31
:102DA0004018606332460599FAF7B2FE0028D7D181
:102DB000606B801960631420D2E71C20D0E700000C
:102DC000F7B58118012349029B0288B0994206D9C0
:102DD0002E4A2FA10020F9F7CFFD0BB0F0BD410224
:102DE0004B09510204914909069136495A0151187B
:102DF0000291039109990191002801D000263BE03E
:102E0000012639E001997001441803990090451892
:102E1000202221462846F5F797FA00282BD0214694
:102E200028460B22F5F790FA002811D00020264FF3
:102E300005907F6823462A4620460221B84701991B
:102E40000098085CE52805D00598002807D012E016
:102E50000120ECE72A4623461046012108E02046DF
:102E6000FAF7F8FB002806D023462A461846002128
:102E7000154C6468A047761C06988642C2D3049A13
:102E800009990298F5F714FBA7E700007D020000FE
:102E90002E2E5C2E2E5C2E2E5C736F757263655C1D
:102EA0006461706C696E6B5C647261672D6E2D6419
:102EB000726F705C7669727475616C5F66732E6395
:102EC00000000000C809002014F1FF1F10B54B00DE
:102ED0000124591C6402A14206D3FF223B3204A103
:102EE0000020F9F749FD10BDC254120A425410BD2A
:102EF0002E2E5C2E2E5C2E2E5C736F757263655CBD
:102F00006461706C696E6B5C647261672D6E2D64B8
:102F1000726F705C7669727475616C5F66732E6334
:102F200000000000F0B587B0002416460F460546A5
:102F3000039404940594FF2004AA03A9013002928B
:102F4000019100906B1C05AA31463846FBF70EFE36
:102F500000280DD0022814D001281FD0042829D021
:102F6000052801D00628E6D1052825D0012024E037
:102F7000049A002A27D0691C0398FAF7C9FD044671
:102F800021E0049A002A05D0691C0398FAF7C0FDD5
:102F9000040018D10598361A3F18CCE7049A002A85
:102FA00004D0691C0398FAF7B3FD0446002C0AD13B
:102FB000132408E0152406E00020FF22613203A15B
:102FC000F9F7DAFC1624204607B0F0BD2E2E5C2E51
:102FD0002E5C2E2E5C736F757263655C6461706C21
:102FE000696E6B5C647261672D6E2D64726F705CCC
:102FF00066696C655F73747265616D2E63000000B5
:1030000070470000904401000100017800000000BA
:1030100000000000000000002CF1FF1F4152544549
:103020004D49535F48544D415254454D495320201A
:10303000202068747470733A2F2F7777772E73700F
:1030400061726B66756E2E636F6D2F617274656D44
:103050006973000000000000000000000000000094
:103060000000000000000000000000000000000060
:1030700000009DED000000000000000000000000C6
:10308000000053544152545F424C414354000000ED
:10309000F84B01009C4B01007C4B0100544C01009B
:1030A00030480100444B010048480100944A0100A7
:1030B000344A0100144C0100F04A0100B8490100F3
:1030C000F44901007C4C0100B44B0100E4480100CC
:1030D000B84801009048010014490100D04A01009D
:1030E000384C010000460100C04501008445010044
:1030F00044490100FC4701005847010020470100F6
:10310000484601002445010058450100F8440100EB
:1031100098440100C8440100B847010098460100E6
:10312000D4460100D04C0100944701006D1101000C
:10313000A9130100D911010071100100E10F010074
:1031400025130100DD100100C10F01005113010022
:103150002C31010030313233343536373839616241
:10316000636465660000000071E300008D190100D2
:103170000DEE0000A5D200000DD2000061EF0000AE
:1031800079D30000D10F0100000000006831010078
:1031900000000000FFFFFFFFFFFFFFFFFFFFFFFF3B
:1031A000FFFFFFFF00000000000000000000000023
:1031B0000000000000000003747970653A2000658B
:1031C00072726F723A20003C21646F63747970658B
:1031D0002068746D6C3E0D0A3C212D2D206D6265BA
:1031E0006420506C6174666F726D205765627369FC
:1031F000746520616E642041757468656E746963DE
:103200006174696F6E2053686F7274637574202DDA
:103210002D3E0D0A3C68746D6C3E0D0A3C6865617C
:10322000643E0D0A3C6D657461206368617273656C
:10323000743D227574662D38223E0D0A3C74697403
:103240006C653E6D626564205765627369746520C4
:1032500053686F72746375743C2F7469746C653E47
:103260000D0A3C2F686561643E0D0A3C626F64790B
:103270003E0D0A3C7363726970743E0D0A77696E85
:10328000646F772E6C6F636174696F6E2E726570F8
:103290006C6163652822405222293B0D0A3C2F7342
:1032A00063726970743E0D0A3C2F626F64793E0D43
:1032B0000A3C2F68746D6C3E0D0A00415353455211
:1032C00054202054585400008230010000000000B7
:1032D000AC4D010001000000B84D010002000000EB
:1032E000A04D010003000000944D01000400000007
:1032F000884D010005000000644D0100060000003B
:103300007C4D010007000000584D0100080000003E
:10331000704D010009000000404D01000A0000004E
:103320004C4D01000B000000D04D0100EC4D0100A0
:10333000DC4D0100E44D0100C44D0100EB3C904D1B
:1033400053443053342E3100020801000220005053
:103350001FF8010001000100000000000000000053
:10336000000029741902274441504C494E4B2D440A
:103370004E444641543136202020FAB8C00705207B
:10338000018ED0BC0010B8C0078ED8BE6D00E80B0F
:1033900000EBFEB40EB700B307CD10C38A04460895
:1033A000C07405E8EDFFEBF4C3504C454153452094
:1033B00052454D4F5645205448452041524D204DD1
:1033C000424544204441504C494E4B2055534220E5
:1033D00044455649434520414E44205245424F4FB3
:1033E00054205448452053595354454D2E2E000027
:1033F00000000000000000000000000000000000CD
:1034000000000000000000000000000000000000BC
:1034100000000000000000000000000000000000AC
:10342000000000000000000000000000000000009C
:10343000000000000000000000000000000000008C
:10344000000000000000000000000000000000007C
:10345000000000000000000000000000000000006C
:10346000000000000000000000000000000000005C
:10347000000000000000000000000000000000004C
:10348000000000000000000000000000000000003C
:10349000000000000000000000000000000000002C
:1034A000000000000000000000000000000000001C
:1034B000000000000000000000000000000000000C
:1034C00000000000000000000000000000000000FC
:1034D00000000000000000000000000000000000EC
:1034E00000000000000000000000000000000000DC
:1034F00000000000000000000000000000000000CC
:1035000000000000000000000000000000000000BB
:1035100000000000000000000000000000000000AB
:10352000000000000000000000000000000000009B
:103530000000000000000000000055AAA5F20000F5
:10354000013001000002000031F0000001300100F4
:103550000000000031F00000013001000000000018
:10356000B1EF0000C12D01000004000000000000C8
:103570000000000000000028000000000000000023
:103580000000418EBB32000000000000000000007F
:1035900000000000000000010000000076487648AE
:1035A0000000DC83764800000000000000BE0AE056
:1035B0000D782D0668400824400000D35840641E52
:1035C000FAD1491C521E002AF2D170474FF0402018
:1035D00047218161002141618161084670470020D7
:1035E00070472DE9F041334E0025334F06244E44F9
:1035F000224673680021384698470543641C402CD6
:10360000F6DB32680121384690472843BDE8F08157
:1036100010B5C10C00D00121264A4A445368C0F3BA
:10362000453225489847002800D0012010BD2DE9DB
:10363000F04707461646880700D0012000EB9104AA
:10364000DFF8708047EA0600DFF86CA08007C84406
:1036500025D000201FE0B4F5007F01D2A50001E0D5
:103660004FF4006515490020494404E016F8012B89
:1036700001F8012B401CA842F8D31049D8F808C023
:10368000AB0827F0030249445046E047002804D124
:10369000A4EB95042F44002CDDD1BDE8F087D8F8C9
:1036A000085023463A4631465046AC46BDE8F047FE
:1036B0006047000004000000214334122400000091
:1036C000000000004D0000085100000855000008EF
:1036D000590000085D00000861000008650000084E
:1036E0006900000800000000000000000000000069
:1036F00000000000000000000000000000000000CA
:1037000000000000000000000000000000000000B9
:1037100000000000000000000000000000000000A9
:103720000000000000000000000000000000000099
:103EE0000000000000C000000020000021000010C1
:103EF0003300001037000010650000108300001030
:103F00000000000001000010140100100004001067
:103F1000000A00100000001038090000AC35010054
:103F200000200000017802000400000000000000F2
:103F3000000000000000000000000000FD0701007C
:103F40000000000000000000000000000000000071
:103F500008001000180020003000400060008000C1
:103F6000C000000180010002000300040006000000
:103F700001400101010040004000400001014000FB
:103F800040000202400000024000040440004000E3
:103F900040004000212005054000000240000000D4
:103FA00061C7000000000000000000007DC70000A5
:103FB00000000000E5A6000035AE0000A1B500003D
:103FC00057A300003DA30000F9A00000000000007E
:103FD00000000000000000000000000000000000E1
:103FE00000000000000000000000000000000000D1
:103FF0000000000007A60000000000000000000014
:104000000600FF0901A101150026FF007508954073
:104010000901810295400901910295010901B1024E
:10402000C000210012011002EF020140280D04021D
:104030000010010203010000050F390002181005ED
:104040000038B60834A909A0478BFDA0768815B6BC
:1040500065000121001C100500DF60DDD88945C71F
:104060004C9CD2659D9E648A9F000003064A0120F5
:104070000000040309040803410052004D004603F8
:1040800053007000610072006B00460075006E0006
:10409000200041007200740065006D00690073002B
:1040A000200044006500760020004B006900740089
:1040B000200043004D005300490053002D004400F0
:1040C000410050001A033000300030003100410040
:1040D000300030003000300030003000300022036B
:1040E0006D006200650064002000530065007200EE
:1040F000690061006C00200050006F0072007400C5
:1041000022036D006200650064002000530065001A
:104110007200690061006C00200050006F007200A6
:1041200074001A0343004D005300490053002D0052
:104130004400410050002000760031002403570065
:10414000650062005500530042003A002000430021
:104150004D005300490053002D0044004100500021
:1041600010035500530042005F004D005300430010
:104170001A0343004D005300490053002D00440032
:10418000410050002000760032000000080B0002C1
:1041900002020104090400000102020104052400D6
:1041A0001001052401030204240206052406000070
:1041B0000705830310002009040000020A0000051F
:1041C00007050402400000070584024000000400C7
:1041D00088000401FF5207000100000010270000C2
:1041E00000000000CC000000980000000400000067
:1041F00000000000000001010100000001000100BA
:1042000000000000000000000000000000000000AE
:10421000000000000000000000000000000000009E
:104220000000000000000000020002000100000089
:10423000000000000000000000000000000000007E
:10424000000000000000000000000000000000006E
:104250000000000003000200040000000000000055
:10426000000000000000000000000000000000004E
:10427000000000000000000000000000000000003E
:10428000000000000000000000000000000000002E
:10429000000000000000000000000000000000001E
:104490004131323700000000496E206170706C6954
:1044A000636174696F6E2070726F6772616D6D69A0
:1044B0006E6720736563746F722065726173652027
:1044C0006661696C65642E00496E206170706C696C
:1044D000636174696F6E2070726F6772616D6D6970
:1044E0006E67206D6173732065726173652066610C
:1044F000696C65642E000000496E206170706C6903
:10450000636174696F6E2070726F6772616D6D693F
:104510006E67207772697465206661696C65642EC8
:1045200000000000496E206170706C6963617469FD
:104530006F6E2070726F6772616D6D696E67206952
:104540006E697469616C697A6174696F6E20666105
:10455000696C65642E000000496E206170706C69A2
:10456000636174696F6E2070726F6772616D6D69DF
:104570006E6720756E696E6974206661696C65642A
:104580002E000000546865206865782066696C65B7
:104590002063616E6E6F742062652070726F677247
:1045A000616D6D65642E204C6F676963206661697B
:1045B0006C757265206F636375727265642E00009E
:1045C000546865206865782066696C652063616E53
:1045D0006E6F74206265206465636F6465642E206D
:1045E000506172736572206C6F67696320666169E0
:1045F0006C757265206F636375727265642E00005E
:10460000546865206865782066696C652063616E12
:104610006E6F74206265206465636F6465642E202C
:10462000436865636B73756D2063616C63756C6162
:1046300074696F6E206661696C757265206F636363
:1046400075727265642E0000546865206170706C2C
:1046500069636174696F6E2066696C6520666F724C
:104660006D617420697320756E6B6E6F776E20615B
:104670006E642063616E6E6F74206265207061727B
:1046800073656420616E642F6F722070726F636552
:10469000737365642E000000496E206170706C6950
:1046A000636174696F6E2070726F6772616D6D699E
:1046B0006E67206E6F7420737570706F72746564AE
:1046C000206F6E2074686973206465766963652E57
:1046D00000000000496E206170706C69636174694C
:1046E0006F6E2070726F6772616D6D696E672066A4
:1046F00061696C65642062656361757365207468C7
:1047000065207570646174652073656E74207761CF
:104710007320696E636F6D706C6574652E000000A8
:10472000546865207374617274696E672061646493
:104730007265737320666F722074686520696E7489
:104740006572666163652075706461746520697364
:104750002077726F6E672E005468652073746172E3
:1047600074696E67206164647265737320666F722A
:104770002074686520626F6F746C6F61646572206D
:104780007570646174652069732077726F6E672E2F
:104790000000000054686520626F6F746C6F616484
:1047A00065722043524320646964206E6F742070E8
:1047B0006173732E00000000496E206170706C6997
:1047C000636174696F6E2070726F6772616D6D697D
:1047D0006E672061626F7274656420647565207411
:1047E0006F20616E206F7574206F6620626F756E2A
:1047F000647320616464726573732E00546865206D
:104800006865782066696C65206F666673657420DC
:104810006C6F6164206164647265737320697320D6
:104820006E6F7420636F72726563742E00000000F7
:10483000546865207472616E736665722074696D68
:104840006564206F75742E0046696C652073656E13
:1048500074206F7574206F66206F726465722062B9
:10486000792050432E20546172676574206D69670A
:104870006874206E6F742062652070726F67726159
:104880006D6D656420636F72726563746C792E0060
:10489000466C61736820616C676F726974686D2023
:1048A000777269746520636F6D6D616E6420464137
:1048B000494C555245000000466C61736820616C9C
:1048C000676F726974686D20657261736520616CD1
:1048D0006C20636F6D6D616E64204641494C55528A
:1048E00045000000466C61736820616C676F7269F7
:1048F00074686D20657261736520736563746F728F
:1049000020636F6D6D616E64204641494C55524580
:1049100000000000466C61736820616C676F72690B
:1049200074686D207772697465207665726966793E
:1049300020636F6D6D616E64204641494C55524550
:1049400000000000546865206865782066696C6521
:1049500020796F752064726F707065642069736E62
:10496000277420636F6D70617469626C652077696C
:1049700074682074686973206D6F6465206F72209D
:104980006465766963652E2041726520796F7520B4
:10499000696E204D41494E54454E414E4345206D70
:1049A0006F64653F205365652048454C5020464163
:1049B000512E48544D00000054686520696E74659E
:1049C0007266616365206669726D77617265204603
:1049D00041494C454420746F20696E697469616C6B
:1049E000697A652074686520746172676574204D0A
:1049F0004355000054686520696E74657266616392
:104A000065206669726D77617265204641494C4543
:104A10004420746F20756E696E697469616C697A7F
:104A2000652074686520746172676574204D435514
:104A30000000000054686520696E746572666163E9
:104A400065206669726D77617265204641494C4503
:104A50004420746F20646F776E6C6F61642074689B
:104A60006520666C6173682070726F6772616D6D2E
:104A7000696E6720616C676F726974686D7320740A
:104A80006F2074686520746172676574204D4355AA
:104A90000000000054686520696E74657266616389
:104AA00065206669726D77617265204641494C45A3
:104AB0004420746F2072657365742F68616C742074
:104AC00074686520746172676574204D43550000F9
:104AD000456E64206F662073747265616D20686135
:104AE00073206265656E20726561636865640000AD
:104AF00054686520696E74657266616365206669D5
:104B0000726D77617265204641494C454420746F4F
:104B100020646F776E6C6F61642074686520666CCA
:104B2000617368206461746120636F6E74656E7474
:104B30007320746F2062652070726F6772616D6D93
:104B400065640000506F737369626C65206D6973F2
:104B50006D61746368206265747765656E2066694F
:104B60006C652073697A6520616E642073697A656B
:104B70002070726F6772616D6D656400416E2069AF
:104B80006E7465726E616C206572726F72206861FE
:104B900073206F636375727265640000416E2065F7
:104BA00072726F7220686173206F636375727265D1
:104BB0006400000054686520696E74657266616304
:104BC00065206669726D77617265204641494C4582
:104BD0004420746F20756E6C6F636B207468652061
:104BE00074617267657420666F722070726F67728D
:104BF000616D6D696E6700004F7065726174696FF9
:104C00006E20776173207375636365737366756C6B
:104C10000000000054686520666C61736820616C58
:104C2000676F206D697373696E6720666F722061AC
:104C300020726567696F6E00456E64206F66207331
:104C4000747265616D20697320756E6B6E6F776E1F
:104C500000000000416E206572726F72206F636306
:104C6000757272656420647572696E672074686518
:104C7000207472616E73666572000000546865206E
:104C8000696E74657266616365206669726D7761CD
:104C900072652041424F525445442070726F6772D2
:104CA000616D6D696E672E20496D6167652069735E
:104CB00020747279696E6720746F20736574207335
:104CC000656375726974792062697473000000000D
:104CD000000000004120626F6F746C6F6164657248
:104CE00020757064617465207761732073746172DC
:104CF0007465642062757420756E61626C652074E1
:104D00006F20636F6D706C6574652E0D0A52656C53
:104D10006F61642074686520626F6F746C6F61648A
:104D2000657220746F2066697820746869732065E5
:104D300072726F72206D6573736167652E0D0A0064
:104D40004D53445F4F4E2020434647004D53445F30
:104D50004F464620434647004F56464C5F4F4E2035
:104D6000434647004155544F5F4F4E20434647004E
:104D70004F56464C5F4F4646434647004155544FB9
:104D80005F4F464643464700484152445F525354A2
:104D9000434647004155544F5F52535443464700E2
:104DA000455241534520202041435400415353452F
:104DB0005254202041435400524546524553482006
:104DC00041435400696E746572666163650000005A
:104DD000696E7465726E616C0000000075736572B7
:104DE0000000000074617267657400007472616E87
:104DF0007369656E740000004D42454420202020F8
:104E00005646532020202020202020202020202013
:104E1000302E3100344E010000F0FF1FF00500007D
:104E20000A880000B04F0100F0F5FF1F903200002B
:104E30000481000021380801010206020208013A3B
:104E400004062F010106060604017A10010523015C
:104E5000999697E401010102270423EBD12375E918
:104E600014292D0123B9CC1AFD101A7D1014252FF9
:104E7000011AC110018814E43E0139E342C04A100E
:104E80000C311AEC1801B722101A060401CF846CF9
:104E9000DC021206126B520A1603064A010829198F
:104EA00012A012141203A757494E555342128412EE
:104EB000041207122A12441265127612691A630844
:104EC0001249126E1A7408127212663A611212476F
:104ED0001A5516124432731250127B1239123212C2
:104EE00043124512361A340412321A2D1212431A82
:104EF00037023A2D121A461C29141A33021A420A92
:104F000012331A31203A422612351A410229181258
:104F100039527D0950A01A430C3A4264296E1A4452
:104F2000823A328E298C29A01A360C5A2D881A36CC
:104F30000A3A310C3A451C29043A33CC5A36A0219E
:104F400014F84D0140292C03016F732E6D626564C6
:104F50002E636F6D2F7765627573622F6C616E645F
:104F6000696E672D706167652F3F6269643DCA1382
:104F70002C01251A5501013814FC41011428420165
:104F80001A54041A80041AAC041AD80414044301F5
:104F90001A30041A5C041A88041AB4041AE00414BF
:104FA0000C44011A38041A640404DD243F01000093
:104FB000FFFFFFFFFFFFFFFFFFFFFFFFFFFFFFFF01
:104FC000FFFFFFFFFFFFFFFFFFFFFFFFFFFFFFFFF1
:104FD000FFFFFFFFFFFFFFFFFFFFFFFFFFFFFFFFE1
:104FE000FFFFFFFFFFFFFFFFFFFFFFFFFFFFFFFFD1
:10FBF000FFFFFFFFFFFFFFFFFFFFFFFF417439F132
:00000001FF
